:020000040800F2
:10000000081A0120D9010008E10100089F2B00080F
:10001000552F0008930900089938000800000000D7
:10002000000000000000000000000000EB010008DC
:10003000ED01000800000000EF010008C12F0008DA
:10004000F3010008F3010008F3010008F3010008C0
:10005000F3010008F3010008510A0008F301000849
:10006000F3010008F3010008F3010008F3010008A0
:10007000F3010008F3010008F3010008F301000890
:100080009D090008A9090008F3010008F301000810
:10009000F3010008F3010008F3010008590A000801
:1000A000F3010008F3010008F3010008F301000860
:1000B000F3010008C1300008F3010008F301000853
:1000C000F3010008F3010008F3010008F301000840
:1000D000F3010008813800088D380008F30100089A
:1000E000F3010008F3010008F3010008F301000820
:1000F000F3010008F3010008F3010008F301000810
:10010000F3010008F3010008F3010008F3010008FF
:10011000F3010008F3010008CD300008F3010008E6
:10012000F3010008F3010008B5090008F301000815
:10013000C10900080000000000000000F3010008F1
:10014000F3010008F3010008F3010008F3010008BF
:10015000CD090008F3010008D9090008F3010008DF
:10016000F3010008F3010008F3010008F30100089F
:10017000F3010008F3010008F3010008000000008B
:1001800000000000F3010008000000000000000073
:10019000F30100080000000000000000F301000867
:1001A000000000000000000000000000F301000853
:1001B000F3010008F3010008F3010008F30100084F
:1001C000F3010008DFF80CD000F0A6FB0048004760
:1001D000495A0008081A0120064880470648004787
:1001E000FEE7FEE7FEE7FEE7FEE7FEE7FEE7FEE7E7
:1001F000FEE7FEE769300008C50100080649074A26
:100200000868504343F239021044086040087047C0
:100210000149086070470000080200206D4EC64189
:1002200040EA01039B0703D009E008C9121F08C078
:10023000042AFAD203E011F8013B00F8013B521EF8
:10024000F9D27047D2B201E000F8012B491EFBD26F
:1002500070470022F6E710B513460A4604461946D1
:10026000FFF7F0FF204610BD421C10F8011B0029CB
:10027000FBD1801A704710B5002200E0521C835C4D
:100280008C5CA34201D1002BF8D1D8B2E1B2401A64
:1002900010BD034611F8012B00F8012B002AF9D1FB
:1002A000184670472DE9FE4F804681EA0300C00FD3
:1002B0000C46009021F0004123F00045B8EB02000D
:1002C000A94105D24046214690461C460B460246AF
:1002D00023F00040104347D0270DC7F30A00C3F3B3
:1002E0000A510290401A019040286BDAC3F31300C0
:1002F00040F4801B0098924620B10023D2EB030A01
:1003000063EB0B0B01985946C0F14002504600F0D8
:10031000BDF906460D4650465946019A00F0D5F9FA
:1003200010EB08006141002487EA115284EAE77368
:100330001A4340D0009A62B3019A012A4FEA075249
:1003400015DC001B61EB02014FF0004202EA07528C
:10035000CDE90042001C41F5801132462B4600F0E9
:100360000CFA03B0BDE8F08F40462146F9E7001BC8
:1003700061EB0201001C41F5801300185B4120185D
:10038000A2F5001747EB030140EAD570B6196D419D
:1003900011E06D084FEA360645EAC0754FEA07528C
:1003A000001B61EB0201001C41F5801149084FEA76
:1003B00030000019514132462B4603B0BDE8F04FE2
:1003C00000F0CCB90098012240000023D0EB0202DB
:1003D00063EBE073009821464FEAE074B8EB00004D
:1003E00061EB0401E9E783F000435BE781F0004142
:1003F00058E72DE9FE4F81EA030404F0004421F0A0
:10040000004100944FF0000B23F0004350EA010438
:100410005ED052EA03045BD0C3F30A54C1F30A5519
:100420002C44A4F2F3340194A0FB0254C1F3130151
:1004300041F48011C3F3130343F4801301FB02441E
:1004400000FB034E840A970A44EA815447EA835723
:10045000A4FB076802958D0A05FB07854FEA932CDC
:1004600004FB0C542705029D4FEA065847EA16374D
:10047000B5EB08056EEB070C870E920E47EA811765
:1004800042EA8312A7FB0201B6EB0B0164EB000406
:100490002B0D43EA0C335E1844EB1C50DA465146F0
:1004A000E7FB0201C5F313044FEA0B3343EA14538D
:1004B0004FEA0432019C43EA0603A4F10C040294BF
:1004C000009CCDE900B400F058F903B0BDE8F08F0E
:1004D00000200146F9E72DE9F04D81EA030404F01C
:1004E000004B21F0004514464FF0000A23F0004174
:1004F00050EA050220D054EA01021DD0C5F30A5784
:100500000246C5F31303C1F31300C1F30A5640F4C6
:10051000801543F48013A7EB0608101BD64608F29B
:10052000FD3873EB050002D308F1010801E09218D1
:100530005B41B8F1000F03DA00200146BDE8F08D01
:1005400000204FF48011064684460EE0171B73EB23
:10055000050705D3121B63EB050306434CEA010CA8
:1005600049084FEA300092185B4150EA0107EDD18B
:1005700052EA030012D082EA040083EA050108432C
:1005800005D0101BAB4106D20122002306E0002259
:100590004FF0004302E06FF0010253101AEB060027
:1005A0004CEB085110EB0A0041EB0B01BDE8F04D9C
:1005B00000F0D4B80EB5C10F80EAE0700844CA0755
:1005C000002140F233438DE80E000A460B4600F04E
:1005D000D4F803B000BD0EB540F2334102910021C2
:1005E000CDE900110A460B4600F0C7F803B000BD84
:1005F00070B5C1F30A5201F000450024C1F31301A4
:1006000040F2FF3341F480119A4201DA002070BDBC
:1006100040F233439A42A2F2334203DC524200F0EA
:1006200044F800E090402C43F1D0404270BD00F00F
:10063000004230F000400AD0C10D01F56071C0F3F6
:10064000160042EA0151C2084007114370470020DA
:100650000146704701F0004330B421F0004150EAF8
:10066000010206D00A0DA2F56072C1F31301002A3F
:1006700002DC30BC00207047440F44EAC104C100D2
:10068000E01830BC00EBC25000F031B8202A04DB87
:10069000203A00FA02F1002070479140C2F1200395
:1006A00020FA03F3194390407047202A04DB203AD4
:1006B00021FA02F00021704721FA02F3D040C2F182
:1006C00020029140084319467047202A06DBCB17C9
:1006D000203A41FA02F043EAE07306E041FA02F3FD
:1006E000D040C2F1200291400843194670470029CA
:1006F000A8BF7047401C490008BF20F001007047A8
:1007000010B4B0FA80FC00FA0CF050EA010404BF07
:1007100010BC704749B1CCF1200421FA04F411FA5D
:100720000CF118BF012121430843A3EB0C01CB1DA1
:100730004FEA00614FEA102042BF002010BC704712
:1007400000EBC35010440029A4BF10BC7047401CEC
:10075000490008BF20F0010010BC704710B5141EFE
:1007600073F1000408DA401C41F1000192185B416A
:100770001A4301D120F0010010BD2DE9F04D924641
:100780009B4611B1B1FA81F202E0B0FA80F2203258
:100790009046FFF77BFF04460F4640EA0A0041EA15
:1007A0000B0153465A46084313D0114653EA010041
:1007B00019D0C8F140025046FFF777FF05460E46B4
:1007C000504659464246FFF761FF084305D00120D5
:1007D00004E020463946BDE8F08D0020054346EA96
:1007E000E0762C4337430A986305E40AA0EB08003F
:1007F0000022FD0A44EA47540A3002D5002001468F
:10080000E9E7010510196941DDE908450019694169
:10081000BDE8F04DA2E72DE9F04D00231A461B1A62
:100820008A4103DB00200146BDE8F08DC1F30A5286
:10083000C1F3130141F480154FF0000BD10702D131
:1008400000186D41521E0027044640F2FF11384641
:1008500001EB620A3E468046024600204FF48011BA
:10086000FFF723FFC2197141BB1846EB0100B4EB3F
:10087000030C75EB000C04D3E41A65EB0005174676
:100880000E46241908F101006D4180463428E3DD4D
:10089000F91946EB0600091BA84103D24FF0FF32BD
:1008A000134601E0002213461BEB070046EB0A51FA
:1008B000BDE8F04DFFF752BF30B5041E71F10004E2
:1008C00004DB4FF00044404264EB0101141E73F15D
:1008D000000405DB1C464FF00043524263EB040367
:1008E0008B4208BF824230BD30B5041E71F1000456
:1008F00004DB4FF00044404264EB0101141E73F12D
:10090000000405DB1C464FF00043524263EB040336
:10091000994208BF904230BD064C074D06E0E068A2
:1009200040F0010394E8070098471034AC42F6D336
:10093000FFF74CFC287700084877000870B58C1842
:1009400010F8015B15F0070301D110F8013B2A11E3
:1009500006D110F8012B03E010F8016B01F8016BD0
:100960005B1EF9D12B0705D40023521E0DD401F8CC
:10097000013BFAE710F8013BCB1A921C03E013F895
:10098000015B01F8015B521EF9D5A142D8D30020CA
:1009900070BD0B2003F03AFFFEE70000014800F0B5
:1009A000E3B90000DCCA0020014800F0DDB9000016
:1009B00084CA0020014800F0D7B900006405002077
:1009C000014800F0D1B900000C050020014800F0FA
:1009D000CBB90000D4C90020014800F0C5B900001F
:1009E0002CCA002001680A4BCAB2103AA3FB02329B
:1009F0001209084B9B5C4365032A04D96FF3090174
:100A0000091D016502E06FF309010165006D704782
:100A1000ABAAAAAA1873000810B4D0F800C0DCF87A
:100A2000004024F48024CCF80040D0F800C0CCF87A
:100A300004308368402B05D0036899600068C26069
:100A400010BC704703689A600068C16010BC7047B2
:100A5000012000F099BC000010B504F07FF80649B1
:100A60000020086005490860054980204861BDE80C
:100A70001040402000F088BC1408024014040240DA
:100A8000000002400022002905D001291FD00229C0
:100A900020D04FF4407211490B6823F440730B606F
:100AA0000B681A430A600A6822F0F8020A600A68B2
:100AB000F82393FAA3F3B3FA83F3984040F00200CB
:100AC00010430860086840F48030086070474FF4B5
:100AD0008072E0E74FF40072DDE70000103C024056
:100AE0001448016811F4007F0FD0016821F40071EF
:100AF0000160016841F400610160016821F4006156
:100B00000160016841F400710160016811F4806FB7
:100B10000FD0016821F480610160016841F48051C7
:100B20000160016821F480510160016841F4806135
:100B300001607047003C02400748016821F44071A1
:100B4000016001680160016841F004010160016811
:100B500041F4803101607047103C0240064A13683E
:100B600023F44073136013681360136843F00103A8
:100B70001360017070470000103C02400A49D1F830
:100B800000C02CF4407CC1F800C0D1F800C04CF487
:100B9000407CC1F800C0D1F800C04CF0010CC1F895
:100BA00000C0026043607047103C0240074A13686F
:100BB00023F440731360136843F480731360136865
:100BC00043F001031360018070470000103C0240B5
:100BD000074A136823F440731360136843F40073E7
:100BE0001360136843F00103136001607047000055
:100BF000103C02401F49086810F0100F1E4805D035
:100C0000C26942F01002C26110220A600A6812F042
:100C1000200F05D0C26942F00802C26120220A609A
:100C20000A6812F0400F05D0C26942F00402C261A6
:100C300040220A600A6812F0800F05D0C26942F0B3
:100C40000202C26180220A600A6812F4807F06D024
:100C5000C26942F00102C2614FF480720A600A6800
:100C600012F0020F05D0C26942F02002C2610220D8
:100C7000086070470C3C0240E8F9002070B504465B
:100C800014490020C86100F0A3FC0646124D2868F4
:100C900010F4803F0ED0B4F1FF3F07D024B100F034
:100CA00097FC801BA04201D9032070BD286810F476
:100CB000803FF0D1286810F0010F01D0012028609A
:100CC000286810F4F97F03D0FFF794FF012070BD6E
:100CD000002070BDE8F900200C3C024002F04EF903
:100CE0000121084600F080FDBFF34F8F05480168E1
:100CF000054A01F4E06111430160BFF34F8F00BF6B
:100D0000FDE700000CED00E00400FA0570B50446B4
:100D10002068016821F00101016000F059FC0546DE
:100D2000206800684FF0000610F0010F14D000F0AA
:100D30004FFC401BB0F57A7F09D9E06C40F02000F1
:100D4000E06484F83460032084F8350070BD2068C6
:100D5000006810F0010FEAD184F83460012084F8B3
:100D60003500002070BD00002DE9F0410446256DDE
:100D7000286894F85420082101FA02F210424FF03A
:100D800004074FF0000619D02068026812F0040F23
:100D900014D0026822F00402026094F8540001FAB0
:100DA00000F0A860E06C40F00100E06484F8357069
:100DB00084F83460A16C09B120468847286894F80B
:100DC00054205F4901FA02F2104219D020684269AA
:100DD00012F0800F14D0426922F08002426194F830
:100DE000540001FA00F0A860E06C40F00200E064FA
:100DF00084F8357084F83460A16C09B120468847C6
:100E0000286894F854204F4901FA02F2104219D090
:100E10002068026812F0020F14D0026822F0020269
:100E2000026094F8540001FA00F0A860E06C40F011
:100E30000400E06484F8357084F83460A16C09B172
:100E400020468847286894F85410102202FA01F1CD
:100E500008422ED02068036813F0080F29D00368D9
:100E600013F4802F4FF0310310D0A960206801687F
:100E700011F4002F07D0006810F4002F15D0412086
:100E800084F8350011E084F835300EE0016811F483
:100E9000807F03D1016821F00801016094F85400BB
:100EA00002FA00F0A86084F83530216C09B12046C0
:100EB0008847286894F85410202202FA01F1084269
:100EC0003BD02068036813F0100F36D0036813F48A
:100ED000802F17D0A9602068016811F4002F0AD074
:100EE000006810F4002F28D0E16B002925D020469F
:100EF000BDE8F0410847616C00291ED02046BDE8DE
:100F0000F0410847016811F4807F03D1016821F0A6
:100F10001001016094F8540002FA00F0A860E06C3F
:100F2000E064112084F8350084F83460E16B002916
:100F300003D02046BDE8F0410847BDE8F08100003D
:100F4000010080000400800070B50446002C27D00A
:100F5000616A022084F83500226810681E4B184030
:100F6000D4F808C06368256943EA0C03D4F80CC0C0
:100F70004CEA050C43EA0C03D4F814C043EA0C0312
:100F8000D4F818C043EA0C03D4F81CC043EA0C039D
:100F9000D4F820C043EA0C031843042902D005E02A
:100FA000012070BD236BE16A194308431060226879
:100FB000506920F00700616A0843042901D1A16A41
:100FC000084350612046FFF70DFD0020E06401203A
:100FD00084F83500002070BD3F8010F02DE9F05FEF
:100FE000044688461646256D606DB8F1000F47D05F
:100FF000102101FA00F700F0EBFA814628684FF063
:10100000000A384258D1DFF838B12A6894F8540001
:101010000821814011402A680BFA00F31A40D5F8E4
:1010200000C0484B03FA00F00CEA000041EA02035A
:10103000034329D041B1E16C41F00101E16494F82E
:10104000543008219940A96042B1E16C41F002019D
:10105000E16494F854100BFA01F1A96040B1E06C1E
:1010600040F00400E06494F8541036488840A860CA
:10107000042084F8350084F834A00120BDE8F09FF6
:10108000202101FA00F7B6E7B6F1FF3F11D02EB1EB
:1010900000F09EFAA0EB0900B0420AD9E06C40F0E3
:1010A0002000E064032084F8350084F834A0BDE813
:1010B000F09F28683842A8D0B8F1000F17D094F8F4
:1010C000541010208840A8602068016811F4802F17
:1010D0004FF031012FD0026812F4002F28D00068A1
:1010E00010F4002F29D0412084F8350025E094F831
:1010F0005400302101FA00F0A8602068016811F462
:10110000802F4FF011010ED0026812F4002F07D08B
:10111000006810F4002F08D0212084F8350004E086
:1011200084F8351001E084F8351084F834A004E028
:1011300084F8351001E084F835100020BDE8F09FF8
:10114000010080000400800010B5044694F83400CB
:10115000012816D0012084F83400022084F83500DC
:101160002068D0F800C02CF0010CC0F800C0204668
:10117000FFF752FC2068016841F001010160002086
:1011800010BD022010BD10B5044694F834000128AB
:1011900020D0012084F83400022084F83500206833
:1011A000D0F800C02CF0010CC0F800C02046FFF7BA
:1011B00033FC2068016841F01E010160206841692C
:1011C00041F0800141612068016841F00101016046
:1011D000002010BD022010BD31B500F0F9F9044621
:1011E00000F0F6F90099001B8842F9D338BD0000E1
:1011F0002DE9F04104460F46DFF8988098F8180072
:1012000001280AD0012088F818004CF25030FFF76E
:1012100035FD0246100003D035E00220BDE8F08124
:101220004FF0FF30386020681B4E012815D0A568AC
:10123000E0682844A84224D9217C2846FFF722FCF4
:101240004CF25030FFF71AFD0246306820F0FA00E9
:10125000306010000FD03D6013E0207C6168FFF724
:101260006BFC4CF25030FFF709FD0246306820F06D
:101270000400306005E06D1CA168E0680844A842E5
:10128000DAD8FFF72DFC002088F818001046BDE8DA
:10129000F0810000E8F90020103C0240034801689A
:1012A00041F000410160002070470000103C024006
:1012B0002DE9F0410646884614461D461A4F387EF1
:1012C000012807D0012038764CF25030FFF7D6FCC9
:1012D00018B115E00220BDE8F081AEB1012E18D0A2
:1012E000022E1BD022462B464046FFF747FC4CF20D
:1012F0005030FFF7C3FC0D490A6822F001020A6072
:1013000000213976BDE8F081E1B24046FFF726FCC6
:10131000EDE7A1B24046FFF749FCE8E72146404629
:10132000FFF756FCE3E70000E8F90020103C02401C
:101330000648006810F0004F06D0064804490160D6
:10134000054901600020704701207047103C0240B1
:1013500023016745043C0240AB89EFCD10B504463C
:1013600014F0010F04D007490120087001F0F6FDC8
:1013700014F0400F05D0BDE8104042F2107004F0A8
:101380002FBD10BD5C01002010B504490A6802425F
:1013900002D00860FFF7E2FF10BD0000143C0140DE
:1013A0002DE9F84F0022DFF8F081DFF8F091DFF847
:1013B000F0A14FF0030E0F27012303FA02F50B688B
:1013C0002B40AB427DD1D1F804C0BCF1020F02D05A
:1013D000BCF1120F12D14FEAD20C00EB8C0CDCF8EE
:1013E00020605407E40E07FA04FB26EA0B06D1F846
:1013F00010B00BFA04F43443CCF8204006684FEAEE
:10140000420C0EFA0CF4A64391F804B00BF0030B57
:101410000BFA0CFB4BEA060606604E68012E05D05F
:10142000022E03D0112E01D0122E11D18668A643B0
:10143000D1F80CB00BFA0CFB4BEA06068660466846
:1014400026EA05050E79C6F3001696403543456039
:10145000C56825EA04048D6805FA0CFC4CEA040C06
:10146000C0F80CC0D1F804C01CF0805F78D0D8F868
:1014700000C04CF4804CC8F800C0D8F800C00CF490
:10148000804CCDF800C022F0030C0CF1804505F52E
:101490009835D5F808C89407240F07FA04F62CEA03
:1014A0000606A0F1804CBCF5003C5FD0A0F1804C5A
:1014B000BCF5013C5DD0A0F1804CBCF5023C5BD09A
:1014C00000E04DE0A0F1804CBCF5033C57D0A0F10A
:1014D000804CBCF5043C55D0A0F1804CBCF5053CDB
:1014E00053D0A0F1804CBCF5063C51D04FF0080C15
:1014F0000CFA04FC4CEA060CC5F808C8D9F800C080
:101500002CEA030C4C6814F4803F01D04CEA030C25
:10151000C9F800C0234CD4F800C02CEA030C4D6875
:1015200015F4003F01D04CEA030CC4F800C01E4C77
:10153000D4F800C02CEA030C4D6815F4801F01D0CC
:101540004CEA030CC4F800C0DAF800C02CEA030C23
:101550004C6814F4001F01D04CEA030CCAF800C018
:10156000521C102AFFF428AFBDE8F88F4FF0000C92
:10157000BEE74FF0010CBBE74FF0020CB8E74FF0AD
:10158000030CB5E74FF0040CB2E74FF0050CAFE7E2
:101590004FF0060CACE7000044380240003C01402C
:1015A0000C3C0140043C0140083C014000690842F9
:1015B00001D00120704700207047426951404161CD
:1015C0007047002A01D0816170470904816170472A
:1015D00001480068704700000402002002480168CA
:1015E000491C0160704700000402002010B50B4840
:1015F000016841F400710160016841F4806101609B
:10160000016841F480710160032000F083F8032039
:1016100000F006F800F015F8002010BD003C024074
:1016200010B5044600F03CFA4FF47A72B0FBF2F0C9
:1016300000F030FD00222146501E00F037F8002057
:1016400010BD10B5032000F065F8002211466FF0C0
:101650000B0000F02BF8002211466FF00A0000F09A
:1016600025F8002211466FF0090000F01FF8002253
:101670000321BDE81040081F00F018B800F01F015A
:10168000012202FA01F14009800000F1E020C0F8D7
:101690008011704700F01F01012202FA01F1400998
:1016A000800000F1E020C0F80011704710B4184B22
:1016B0001B68C3F30223C3F1070CBCF1040F01D96B
:1016C0004FF0040C1C1D072C01D2002300E0DB1E90
:1016D000012404FA0CFCACF1010C0CEA0101994064
:1016E00004FA03F35B1E1A401143002808DA00F0E5
:1016F0000F0000F1E020090180F8141D10BC7047B4
:1017000000F1E020090180F8001410BC70470000CF
:101710000CED00E000F00700064A11684FF6FF03E9
:10172000194041EA002040F0FD7040F080601060F8
:10173000704700000CED00E0F8B52548016841F065
:1017400080510160006800F0805000900126300454
:1017500090FAA0F0B0FA80F0800000F1844000F52B
:1017600060200660FFF734FF05461A4C606810F4ED
:10177000803F0BD1FFF72CFF401BB0F57A7F01D9DA
:101780000320F8BD606810F4803FF3D04FF40030C0
:1017900090FAA0F0B0FA80F0800000F1844000F5EB
:1017A00060200660FFF714FF0546606810F4003FF4
:1017B0000BD1FFF70DFF401BB0F57A7F01D9032055
:1017C000F8BD606810F4003FF3D00020F8BD0000C1
:1017D000403802400070004002494A6822EA000096
:1017E00048607047007000400B4A136823F0030301
:1017F000184310600948026842F00402026001299F
:1018000007D040BF20BF20BF016821F00401016064
:10181000704730BFF8E700000070004010ED00E0B6
:101820002DE9F04704460E46DFF868A2DAF800001A
:10183000994900F00F00994F06F0FF0941F28838EE
:10184000B04270D28AF80090DAF8000000F00F0081
:10185000B04202D00120BDE8F087207810F0020FDE
:1018600005D03868A26820F0F00010433860207876
:1018700010F0010F49D06068012808D002280DD06F
:1018800003280BD0096811F0020F29D00AE009687B
:1018900011F4003F06D10120BDE8F087096811F07E
:1018A000007F1AD0396821F0030108433860FFF740
:1018B0008FFE05466068012815D0022826D003282F
:1018C0003BD0386810F00C0F1FD0FFF781FE401B93
:1018D000404539D90320BDE8F0870120BDE8F087F5
:1018E0000120BDE8F087386800F00C0004280CD017
:1018F000FFF76EFE401B404502D90320BDE8F0878C
:10190000386800F00C000428F2D1A8E0386800F034
:101910000C00082870D0FFF75BFE401B404503D940
:101920000320BDE8F08714E0386800F00C000828B8
:10193000F1D194E00320BDE8F0873868FFF748FE56
:10194000401B4045F9D9F5E7386810F00C0FBCD1C1
:1019500085E0207810F0020F05D03868A26820F0EA
:10196000F00010433860207810F0010F6CD06068F0
:10197000012808D002280DD003280BD0096811F0E7
:10198000020F29D00AE0096811F4003F06D10120B6
:10199000BDE8F087096811F0007F1AD0396821F09E
:1019A000030108433860FFF713FE0546606801280D
:1019B00015D0022827D003283BD0386810F00C0F30
:1019C00042D0FFF705FE401B404539D90320BDE852
:1019D000F0870120BDE8F0870120BDE8F087386876
:1019E00000F00C0004282FD0FFF7F2FD401B40450B
:1019F00003D90320BDE8F08731E0386800F00C001F
:101A00000428F1D120E0386800F00C0008281BD031
:101A1000FFF7DEFD401B404502D90320BDE8F087FB
:101A2000386800F00C000828F2D10DE00320BDE872
:101A3000F0873868FFF7CCFD401B4045F9D9F5E742
:101A4000386810F00C0FBCD18AF80090DAF800006A
:101A500000F00F00B04202D00120BDE8F0872078EE
:101A600010F0040F05D03868E16820F4E050084316
:101A70003860207810F0080F06D03868216920F40B
:101A8000604040EAC10038600320FFF7C9FD002034
:101A9000BDE8F087003C02400038024008380240B0
:101AA00010B500F043F808490968F02292FAA2F252
:101AB00001F0F001B2FA82F2D140044A515CC84010
:101AC0000349086010BD0000083802402073000878
:101AD0000002002010B5FFF7E3FF074909684FF443
:101AE000E05292FAA2F201F4E051B2FA82F2D1404D
:101AF000024A515CC84010BD0838024020730008FB
:101B000010B5FFF7CDFF074909684FF4604292FA1C
:101B1000A2F201F46041B2FA82F2D140024A515C71
:101B2000C84010BD083802402073000810B4354882
:101B3000006810F00C0134481DD0DFF8D0C0042933
:101B400018D0334B47F6C072082916D00C2912D191
:101B5000196801F03F011C6814F4800F39D0BCFBF8
:101B6000F1F01968114092FAA2F2B2FA82F2D14071
:101B7000484338E0604610BC7047196801F03F01E7
:101B80001C6814F4800F0AD0BCFBF1F019681140F6
:101B900092FAA2F2B2FA82F2D140484309E0B0FBD5
:101BA000F1F01968114092FAA2F2B2FA82F2D14031
:101BB000484319684FF4403292FAA2F201F44031DE
:101BC000B2FA82F2D140491C4900B0FBF1F010BCDE
:101BD0007047B0FBF1F01968114092FAA2F2B2FA24
:101BE00082F2D140484319684FF0E04292FAA2F2E3
:101BF00001F0E041B2FA82F2D140B0FBF1F010BC4A
:101C000070470000083802400024F40040787D014D
:101C1000043802402DE9F84F0446DFF83484207878
:101C20004FF0000710F0010F41F28836A8F10405CB
:101C300069D008F10400016801F00C01042912D0F8
:101C4000016801F00C01082904D1D8F8001011F442
:101C5000800F08D101680C2088430DD1D8F800000E
:101C600010F4800F08D0286810F4003F4BD0606853
:101C700078BB0120BDE8F88FDFF8D8A38AF80070A0
:101C8000FFF7A6FC8146286810F4003F0CD0FFF750
:101C90009FFCA0EB0900B04202D90320BDE8F88FF9
:101CA000286810F4003FF2D120798AF800006068BB
:101CB000A8B1FFF78DFC8146286810F4003F22D1BF
:101CC000FFF786FCA0EB0900B04203D90320BDE872
:101CD000F88F18E0286810F4003FF1D013E0FFF708
:101CE00077FC8146286810F4003F0CD0FFF770FCA9
:101CF000A0EB0900B04202D90320BDE8F88F2868A4
:101D000010F4003FF2D12078DFF84C9310F0020F6E
:101D10006CD0D24801684FF0F80B11F00C0F1FD0B7
:101D2000016801F00C01082904D1D8F8001011F461
:101D3000800F15D001680C20884304D1D8F800002A
:101D400010F4800F0CD0E068C8B30120C9F800007F
:101D5000FFF73EFC8246286810F0020F16D022E002
:101D6000286810F0020F05D0E068012802D0012099
:101D7000BDE8F88F28689BFAABF22169B2FA82F2CB
:101D800020F0F8009140084328602FE0FFF720FC86
:101D9000A0EB0A00642802D90320BDE8F88F286868
:101DA00010F0020FF2D028689BFAABF22169B2FA68
:101DB00082F220F0F80091400843286016E0FFE727
:101DC000C9F80070FFF704FC8246286810F0020F83
:101DD0000CD0FFF7FDFBA0EB0A00642802D903201A
:101DE000BDE8F88F286810F0020FF2D1207810F0CB
:101DF000080F34D09A48DFF86CB26169C1B1012193
:101E00000160FFF7E5FB8246DBF8000010F0020FEF
:101E100025D1FFF7DDFBA0EB0A00642802D90320DF
:101E2000BDE8F88FDBF8000010F0020FF1D016E0EB
:101E30000760FFF7CDFB8246DBF8000010F0020FD1
:101E40000DD0FFF7C5FBA0EB0A00642802D90320E0
:101E5000BDE8F88FDBF8000010F0020FF1D1207818
:101E600010F0040F72D08048016841F08051016089
:101E7000006800F080500090DFF8F0B1DBF800005F
:101E800040F48070CBF80000FFF7A2FB8246DBF83D
:101E9000000010F4807F0DD1FFF79AFBA0EB0A0041
:101EA000642802D90320BDE8F88FDBF8000010F4A5
:101EB000807FF1D0DFF8B8B18BF80070FFF788FBB6
:101EC0008246DBF8000010F0020F0DD0FFF780FB18
:101ED000A0EB0A00B04202D90320BDE8F88FDBF87E
:101EE000000010F0020FF1D1207A8BF80000A068FA
:101EF000B0B1FFF76DFB8246DBF8000010F0020F77
:101F000024D1FFF765FBA0EB0A00B04202D9032001
:101F1000BDE8F88FDBF8000010F0020FF1D015E0FB
:101F2000FFF756FB8246DBF8000010F0020F0DD0E1
:101F3000FFF74EFBA0EB0A00B04202D90320BDE838
:101F4000F88FDBF8000010F0020FF1D1A069E0B3C8
:101F50004249096801F00C01082975D0022810D007
:101F6000C9F86070FFF734FB0446286810F0007F62
:101F700066D0FFF72DFB001B64285DD90320BDE868
:101F8000F88FC9F86070FFF723FB0646286810F049
:101F9000007F0BD0FFF71CFB801B642802D90320B5
:101FA000BDE8F88F286810F0007FF3D1216AE0695E
:101FB00047F6C072084392FAA2F2616AB2FA82F25C
:101FC00091404FF0FF33A26A00E039E003EB520288
:101FD0004FF4403393FAA3F3B3FA83F39A401143D7
:101FE00008434FF0706292FAA2F2E16AB2FA82F20A
:101FF000914008434FF0E04292FAA2F2216BB2FA0C
:1020000082F291400843C8F800000120C9F860003E
:10201000FFF7DEFA0446286810F0007F10D1FFF7C2
:10202000D7FA001B642802D90320BDE8F88F28687E
:1020300010F0007FF3D003E0286810F0007F98D103
:102040000020BDE8F88FFFE70120BDE8F88F000011
:10205000043802400238024000004742083802407B
:10206000800E474274380240403802400070004001
:10207000703802404FF0E021042804D0086920F0B5
:10208000040008617047086940F004000861704767
:1020900070470000401EB0F1807F01D301207047DF
:1020A0004FF0E0214861044AF02010700020886160
:1020B000072008610020704723ED00E010B5FFF70E
:1020C000E7FF10BD7047704710B490F83820012A20
:1020D00025D0012280F83820022380F83930D1F849
:1020E00004C00B68CC6843EA0C03D1F808C04CEA82
:1020F000040C43EA0C03D1F810C043EA0C03D1F8F6
:1021000014C0896943EA0C0319430368596480F8D1
:102110003920002180F8381010BC0020704710BC16
:102120000220704710B490F83820012A2AD00123E9
:1021300080F83830022280F839200268D2F804C0D2
:102140002CF0700CC2F804C00268D2F804C00C680D
:102150004CEA040CC2F804C00268D2F808C02CF0A3
:10216000800CC2F808C00268D2F808C049684CEA7E
:102170000101916080F83930002180F8381010BCDE
:102180000020704710BC0220704710B50446002C98
:1021900003D094F8390010B107E0012010BD0020F1
:1021A00084F83800204600F00DF8022084F8390049
:1021B000211D206800F090FF012084F839000020E4
:1021C00010BD00002DE9F84F04464A492068B0F1DF
:1021D000804F69D0A0F18042B2F5806252D0A0F168
:1021E0008042B2F5805269D0A0F18042B2F5A0528F
:1021F00076D0A0F18041B1F5823141D13E480168ED
:1022000041F002010160006800F0020000903C4DC6
:102210003A4828604FF060676F604FF04008C5F89B
:1022200008800026EE604FF48069C5F810904FF4E6
:10223000006AC5F814A04FF4005BC5F818B0EE6151
:102240004FF4403028626E622846FEF77DFEA5629C
:10225000AC632D4D2B4828606F60C5F80880EE6098
:10226000C5F81090C5F814A0C5F818B0EE614FF489
:10227000403028626E622846FEF766FE2562AC6337
:10228000BDE8F88F086840F002000860086800F0B8
:1022900002000090002206211D20FFF707FABDE88A
:1022A000F84F1D20FFF7F6B9086840F001000860FC
:1022B000086800F001000090BDE8F88F086840F061
:1022C00010000860086800F010000090002205214E
:1022D0003620FFF7EBF9BDE8F84F3620FFF7DAB903
:1022E000086840F020000860086800F020000090B6
:1022F000BDE8F88F40380240443802407064024024
:102300000C0500204064024064050020022180F892
:10231000391001680A6842F001020A60012180F860
:1023200039100020704770B5044694F83800012831
:1023300018D0012584F83850022084F8390020682C
:10234000826822F0770222F47F4282600868502877
:102350003AD00EDC20285FD006DC002852D01028AE
:1023600063D154E0022070BD30285AD040285CD19F
:102370003EE0602832D070280CD0B0F5805F03D0EA
:10238000B0F5005F51D113E02068816821F00701AA
:1023900081604AE0CB684A688968206800F00DFFD8
:1023A0002068816821F0770141F0770181603CE08D
:1023B000CB684A688968206800F0FFFE2068816861
:1023C00041F48041816030E0CA684968206800F0CB
:1023D000D7FF5021206800F0FBFE26E0CA6849685C
:1023E000206800F0E0FF6021206800F0F1FE1CE0B2
:1023F000CA684968206800F0C3FF4021206800F0E7
:10240000E7FE12E00021206800F0E2FE0DE010215E
:10241000206800F0DDFE08E02021206800F0D8FEF2
:1024200003E03021206800F0D3FE84F8395000200A
:1024300084F8380070BD704770B5044620680169A3
:102440004FF0000511F0020F17D0C16811F0020F14
:1024500013D0E91E0161012020762068806910F008
:10246000030F03D02046FFF7E6FF05E0204600F00B
:10247000C8F8204600F0E3F825762068016911F0DD
:10248000040F18D0C16811F0040F14D06FF00401CC
:102490000161022020762068806910F4407F03D01B
:1024A0002046FFF7C8FF05E0204600F0AAF82046C6
:1024B00000F0C5F825762068016911F0080F18D0E2
:1024C000C16811F0080F14D06FF0080101610420F9
:1024D00020762068C06910F0030F03D02046FFF774
:1024E000AAFF05E0204600F08CF8204600F0A7F88F
:1024F00025762068016911F0100F18D0C16811F01D
:10250000100F14D06FF010010161082020762068B0
:10251000C06910F4407F03D02046FFF78CFF05E030
:10252000204600F06EF8204600F089F825762068F5
:10253000016911F0010F09D0C16811F0010F05D038
:102540006FF001010161204600F07AF8206801690E
:1025500011F0800F09D0C16811F0800F05D06FF025
:10256000800101612046FFF7ADFD2068016911F08F
:10257000400F09D0C16811F0400F05D06FF0400145
:102580000161204600F078F82068016911F0200F01
:102590000BD0C16811F0200F07D06FF0200101614E
:1025A0002046BDE87040FFF78EBD70BD70B5044693
:1025B00094F8380001280DD0012584F83850022005
:1025C00084F8390042B1042A0AD0082A0CD00C2A17
:1025D00011D10DE0022070BD206800F001FE0AE07C
:1025E000206800F031FE06E0206800F065FE02E0A1
:1025F000206800F099FE84F83950002084F83800F3
:1026000070BD704710B50446002C03D094F8390013
:1026100010B107E0012010BD002084F838002046EA
:1026200000F00CF8022084F83900211D206800F029
:1026300053FD012084F83900002010BD7047704719
:1026400010B5094988420AD108480168491C01604F
:10265000074C207820B100F091FC0020207010BDC4
:10266000044901200870F8E7580400204C010020BC
:102670005C0100205D0100207047704738B50446BA
:102680002168086800F00100CA6802F4807200281E
:1026900007D032B1086848680090E06B40F0010054
:1026A000E0630868C0F340004A6902F0010238B1F3
:1026B00032B1086848680090E06B40F00400E063C5
:1026C0000868C0F38002486900F001003AB130B1F7
:1026D000086848680090E06B40F00200E06308681A
:1026E000C0F3C0004A6902F0010238B132B1086893
:1026F00048680090E06B40F00800E0630868C0F3B1
:102700004010C96801F0200118B111B1204600F055
:10271000ACFE20680168C1F3C011C06800F0800001
:1027200019B110B1204601F005F820680168C1F325
:102730008011C06800F0400019B110B1204600F0CF
:1027400075FEE06B002805D0012084F83900204692
:10275000FFF793FF38BD70B50446002C04D094F801
:102760003900002510B106E0012070BD84F8385012
:10277000204600F021F8022084F839002068C16862
:1027800021F40051C160204600F0C8FE20680169B4
:1027900021F4904101612068416921F02A014161E1
:1027A0002068C16841F40051C160E563012084F8EC
:1027B0003900002070BD00002DE9F04786B00446C6
:1027C00002212068002501224F4B4F02A0F18046D4
:1027D0004FF0070C4FF000684FF480794FF0400A3B
:1027E000B6F5883649D0A0F18046B6F5884641D185
:1027F0004648066846F400360660006800F400307B
:1028000000900C200190029103920491CDF814C025
:1028100001A91846FEF7C4FD3E4E3D483060C6F89B
:102820000480C6F808A0F56037617561B561F5618F
:10283000356275623046FEF787FB2663B463374E18
:1028400035483060C6F80480B560F5603761756161
:10285000B561C6F81C90356275623046FEF774FBB0
:102860006663B463002204212620FEF71FFF2620A2
:10287000FEF710FF06B0BDE8F0872948066846F06D
:1028800010060660006800F0100000904FF4C06071
:102890000190029103920491CDF814C001A9184649
:1028A000FEF77EFD204E1F483060C6F80480B560FC
:1028B000F56037617561B561C6F81C903562756267
:1028C0003046FEF741FB6663B463194E174830602B
:1028D000C6F80480C6F808A0F56037617561B56177
:1028E000F561356275623046FEF72EFB2663B463F0
:1028F000002204212520FEF7D9FE2520FEF7CAFE7E
:1029000006B0BDE8F08700000000024040380240F9
:10291000A060024084CA002088600240DCCA002017
:102920004438024088640240D4C90020B8640240A0
:102930002CCA00202DE9F04104460D46984694F833
:102940003900012804D0122802D00220BDE8F0810D
:102950001DB312B394F83800012821D0012684F861
:1029600038600027E76394F8390012281BD0222032
:1029700084F83900A285E285E08D401EE085A068DC
:10298000B0F5805F13D0434600222021204600F09E
:1029900006FF28B30320BDE8F0810120BDE8F081E7
:1029A0000220BDE8F081322084F83900E2E7434696
:1029B00000222021204600F0F2FE10B10320BDE8E5
:1029C000F081206928B120684068C1B229806D1C5F
:1029D0000EE020684068C0F308012980AD1C07E0C4
:1029E000206998B12068406800F07F0005F8010B6D
:1029F000E08D0028C0D194F8390032280BD084F83B
:102A0000396084F838700020BDE8F08120684068A3
:102A100005F8010BECE7122084F83900F1E700001B
:102A200037B50446134694F83900012804D012281B
:102A300002D003B0022030BD019A52B34BB394F8D8
:102A40003800012828D0012084F83800A262A3852C
:102A50000025E56394F83900122820D0222084F85C
:102A60003900616B1048C863616B10480864616B82
:102A70000F4888642068011D606BFEF784FB2068A6
:102A8000416941F04001416184F8385003B00020B1
:102A900030BD03B0012030BD03B0022030BD322074
:102AA00084F83900DDE70000E9330008233400082A
:102AB000CB330008704770472DE9F04104460D46BE
:102AC000984694F83900012804D0222802D0022028
:102AD000BDE8F0811DB312B394F83800012821D06D
:102AE000012684F838600027E76394F8390022282B
:102AF0001BD0122084F83900A284E284E08C401EAE
:102B0000E084A068B0F5805F13D0434600228021A6
:102B1000204600F044FE08B30320BDE8F081012008
:102B2000BDE8F0810220BDE8F081322084F8390050
:102B3000E2E7434600228021204600F030FE10B13B
:102B40000320BDE8F08128882168C0F308004860B0
:102B5000206908B16D1C05E0AD1C03E0216815F883
:102B6000010B4860E08C0028C8D143460022402178
:102B7000204600F014FE10B10320BDE8F08194F867
:102B80003900322806D084F8396084F83870002083
:102B9000BDE8F081222084F83900F6E77047FF2075
:102BA00001F034BE08B52148016841F4001101600C
:102BB000016801F400110091016841F48001016095
:102BC000006800F480000090002201211020FEF730
:102BD0006DFD1020FEF75EFD002201211120FEF7A1
:102BE00065FD1120FEF756FD002211463A20FEF742
:102BF0005DFD3A20FEF74EFD002211463C20FEF717
:102C000055FD3C20FEF746FD002201214420FEF741
:102C10004DFD4420FEF73EFD002201214620FEF737
:102C200045FDBDE808404620FEF734BD303802407F
:102C3000F0B587B04248016841F0040101600168C5
:102C400001F004010191016841F080010160016817
:102C500001F080010191016841F00101016001680A
:102C600001F001010191016841F002010160016878
:102C700001F002010191016841F008010160006862
:102C800000F0080001904FF40050029000240394DB
:102C900004942C4D02A92846FEF782FB4DF6FF71E5
:102CA0000291012603960494059402A92846FEF792
:102CB00077FB032502950395049402A92248FEF7A9
:102CC0006FFB0296214803900494214F02A93846D5
:102CD000FEF766FB48F6A210029003960494059452
:102CE00002A93846FEF75CFB50200290039404943E
:102CF00002A93846FEF754FB4FF2FF70029003968C
:102D00000494059402A91348FEF74AFB300302908D
:102D10000395049402A93846FEF742FB0420029072
:102D20000395049402A90C48FEF73AFB00221146D1
:102D30000620FEF7BBFC0620FEF7ACFC07B0F0BD9A
:102D40003038024000080240001C02400000111010
:102D50000000024000040240000C024010B586B0A2
:102D60000C484FF080410160002444608460C460DE
:102D70000461FFF70AFA4FF48050029002A9054857
:102D8000FFF7D1FA0094019469460248FFF7CAF9A7
:102D900006B010BDE003002010B586B010480F4902
:102DA00001604FF6FF7141600024846040F26711BA
:102DB000C1604FF400710161FFF7E7F94FF48050F3
:102DC000029002A90648FFF7AEFA00940194694602
:102DD0000348FFF7A7F906B010BD0000000400404B
:102DE0001C04002010B582B00B480A49016042F271
:102DF000283141600024846042F20F71C160FFF706
:102E0000C4F90094019469460348FFF78BF902B0B6
:102E100010BD0000001000405804002010B582B022
:102E20000A480949016059214160002484604FF635
:102E3000FF71C160FFF7A9F9009401946946034846
:102E4000FFF770F902B010BD001400409404002098
:102E500010B594B020481F4901600024446084608C
:102E60004721C16004614461FFF78FF94FF480503E
:102E7000109010A91848FFF756FA1748FFF7C2FB41
:102E80000E940F940EA91448FFF74CF90794089478
:102E900009940A940B944FF400500C900D9407A9D8
:102EA0000D48FFF711F93020009014200190029492
:102EB0000394049405940694002269460648FFF79B
:102EC00075FB1E200190082269460348FFF76EFB40
:102ED00014B010BD00040140D00400200848074988
:102EE00001604FF4E131416000218160C160016106
:102EF0000C2242618161C161FFF72DBC00100140CD
:102F0000BC0500200849074A0A6048600020886024
:102F1000C86008610C224A618861C8610846FFF7F1
:102F20001ABC000000100140BC05002008480749F9
:102F300001604FF4E131416000218160C1600161B5
:102F40000C2242618161C161FFF705BC0044004071
:102F5000FC0500200A2001F059FCFEE70548016845
:102F600021F0010101600449012008600620FEF7FC
:102F700085BB0000003C0140143C014000B585B019
:102F80004FF48070FEF728FC0620FEF777FB012047
:102F90000090094801900020029069460748FEF71A
:102FA000FFF900220A210620FEF780FB0620FEF72B
:102FB00071FB05B000BD00000000111000000240D0
:102FC00010B5FEF70BFBBDE81040FFF777B8000027
:102FD00030B593B02248016841F08051016000682B
:102FE00000F0805000901F48016841F440410160AA
:102FF000006800F4404000900224069401200990EB
:1030000010200A900C9400250D9508200E90B420F5
:103010000F9010941194129406A8FEF7FBFDFEF792
:103020008BFB0D200190029403954FF4A050049067
:10303000E0020590052101A8FEF7F2FBFEF730FD46
:103040004FF47A71B0FBF1F0FFF724F80420FFF79A
:1030500011F803210022081FFEF728FB13B030BD32
:1030600040380240007000400F48016841F4700190
:1030700001600E48016841F0010101600C4A002125
:103080001160026822F4102222F080720260031D97
:10309000084A1A60026822F4802202600648016031
:1030A000064958060860704788ED00E00038024085
:1030B00008380240103000240C38024008ED00E0CF
:1030C0000148FFF7B9B900001C0400200148FFF7D0
:1030D000B3B9000058040020F0B402682B4BDFF8AD
:1030E000B0C02C4D2C4E2D4C98420AD0B0F1804FE0
:1030F00007D0604505D0A84203D0B04201D0A0421D
:1031000003D122F070024F683A43984228D0B0F1C0
:10311000804F25D0604523D0A84221D0B0421FD097
:10312000A0421DD0A0F1804CBCF5A03C18D0A0F16D
:10313000804CBCF5A23C13D0A0F1804CBCF5A43C63
:103140000ED0A0F1804CBCF5C05C09D0A0F1804C41
:10315000BCF5E05C04D0A0F1804CBCF5005C05D16E
:1031600022F44072D1F80CC04CEA020202608A6874
:10317000C2620A688262984201D0A04201D1096904
:10318000016301214161F0BC704700000000014073
:103190000004004000080040000C00400004014012
:1031A00001238B40D0F820C02CEA03030362036A9A
:1031B00002FA01F1194301627047D0F808C02CF4FB
:1031C0007F4C42EA0322114341EA0C0181607047BF
:1031D000826822F07002114341F00701816070475C
:1031E00010B4026A22F001020262036A4268D0F857
:1031F00018C02CF0700C2CF0030C0C6844EA0C0C7A
:1032000023F002038C682343A0F18044B4F580349A
:1032100004D0A0F18044B4F582340DD123F008032A
:10322000CC68234323F0040322F4807222F400725A
:103230004C6922438C6922434260C0F818C0496837
:103240004163036210BC704710B4026A22F010029E
:103250000262036A4268D0F818C02CF4E04C2CF4E7
:10326000407C0C684CEA042C23F020038C6843EA71
:103270000413A0F18044B4F5803404D0A0F180445C
:10328000B4F5823410D123F08003CC6843EA0413F0
:1032900023F0400322F4806222F400624C6942EA87
:1032A00084028C6942EA84024260C0F818C049680E
:1032B0008163036210BC704710B4026A22F480720A
:1032C0000262036A4268D0F81CC02CF0700C2CF02B
:1032D000030C0C6844EA0C0C23F400738C6843EA7A
:1032E0000423A0F18044B4F5803404D0A0F18044DC
:1032F000B4F5823410D123F40063CC6843EA04238C
:1033000023F4806322F4805222F400524C6942EA92
:1033100004128C6942EA04124260C0F81CC0496879
:10332000C163036210BC704710B4026A22F4805279
:103330000262D0F820C04268C36923F4E04323F45A
:1033400040730C6843EA04232CF4005C8C684CEA5C
:10335000043CA0F18044B4F5803404D0A0F1804452
:10336000B4F5823404D122F480424C6942EA8412DA
:103370004260C36149680164C0F820C010BC704756
:10338000036AD0F820C02CF0010CC0F820C0D0F89F
:1033900018C02CF0F00C4CEA021223F00A03194377
:1033A000826101627047036A23F010030362D0F860
:1033B00018C0036A2CF4704C4CEA023223F0A003CC
:1033C00043EA011182610162704710B5806B0021F0
:1033D000C185C184012180F83910C16B41F0100111
:1033E000C163FFF74AF910BD10B50146886B096843
:1033F000096811F4807F0DD10021C18501684A69F7
:1034000022F040024A6190F83910322905D001219A
:1034100080F83910FFF74EFB10BD122180F83910EB
:10342000F8E710B5806BFFF746FB10BD10B50168DB
:10343000CA6822F04002CA6090F83910322910D0D0
:103440000168CA6822F48072CA6001684A6922F081
:1034500001024A61012180F83910FFF79FFB00202B
:1034600010BD222180F83910F7E710B590F8391017
:10347000222903D0322901D0022010BD8168B1F584
:10348000805F11D0016919B30168496801F07F02BA
:10349000816A4B1C83620A70C18D491E0904090CA4
:1034A000C1851CD0002010BD816A02693AB1026852
:1034B0005268D2B20A80816A491C8162ECE70268D4
:1034C0005268C2F308020A80816A891C8162E3E7BC
:1034D00001684A68816A4B1C83620A70DCE70168F4
:1034E000CA6822F02002CA6090F83910322910D040
:1034F0000168CA6822F48072CA6001684A6922F0D1
:1035000001024A61012180F83910FFF7D3FA002047
:1035100010BD122180F83910F7E700002DE9F041C5
:1035200004462068016921F44051E26811430161B9
:103530002068C16821F4037121F414412369A26851
:10354000D4F81CC01A43636943EA0C031A431143BD
:10355000C1602068416921F44071A2691143416151
:10356000E069714A7149724D3226B0F5004F38D08A
:103570002068884201D090427ED1FEF7C1FA00EB6C
:10358000C00101EB001061688900B0FBF1F0A5FB00
:1035900000104709FEF7B4FA00EBC00101EB001080
:1035A00061688900B0FBF1F8FEF7AAFA00EBC001F0
:1035B00001EB001061688900B0FBF1F0A5FB001081
:1035C00040096FF01801484308EB800006EB00103B
:1035D000A5FB00102168400967F31F108860BDE853
:1035E000F0812068884201D0904233D1FEF788FAFA
:1035F00000EBC00101EB001061684900B0FBF1F085
:10360000A5FB00104709FEF77BFA00EBC00101EBB8
:10361000001061684900B0FBF1F8FEF771FA00EBA9
:10362000C00101EB001061684900B0FBF1F0A5FB9F
:10363000001040096FF01801484308EB800006EBCA
:103640000010A5FB00102168400967F31F10886077
:10365000BDE8F081FEF73EFA00EBC00101EB00107F
:1036600061684900B0FBF1F0A5FB00104709FEF7C7
:1036700031FA00EBC00100E022E001EB00106168CC
:103680004900B0FBF1F8FEF725FA00EBC00101EBB1
:10369000001061684900B0FBF1F0A5FB0010400983
:1036A0006FF01801484308EB800006EB0010A5FB03
:1036B00000102168400967F31F108860BDE8F081A1
:1036C000FEF708FA00EBC00101EB00106168890009
:1036D000B0FBF1F0A5FB00104709FEF7FBF900EB8A
:1036E000C00101EB001061688900B0FBF1F8FEF742
:1036F000F1F900EBC00101EB001061688900B0FB3B
:10370000F1F0A5FB001040096FF01801484308EBE9
:10371000800006EB0010A5FB00102168400967F34C
:103720001F108860BDE8F0810014014000100140C6
:103730001F85EB5190F83910122903D0322901D09E
:10374000022070478168B1F5805F0CD0016A4A1C85
:103750000262026809785160C18C491E0904090C93
:10376000C18410D019E0016A02680988C1F3080118
:103770005160016919B1016A491C0162ECE7016AF3
:10378000891C0162E8E70168CA6822F08002CA6009
:103790000068C16841F04001C160002070472DE918
:1037A000F04704460E4692461D46FDF711FF0746B8
:1037B0004FF000084FF00109BAF1000F05D0206862
:1037C000006836EA00002FD057E02068006836EA2B
:1037D000000052D0B5F1FF3F20D025B1FDF7F8FE33
:1037E000C01BA8421AD92068C16821F08001C160BD
:1037F0002068C16821F02001C1602068C16821F4FF
:103800008071C1602068416921F00101416184F843
:10381000399084F838800320BDE8F087206800687C
:1038200036EA0000D6D128E0B5F1FF3F20D025B11F
:10383000FDF7CEFEC01BA8421AD92068C16821F04E
:103840008001C1602068C16821F02001C16020684A
:10385000C16821F48071C1602068416921F00101D3
:10386000416184F8399084F838800320BDE8F087FE
:103870002068006836EA0000D6D00020BDE8F08756
:103880000148FEF7FBBE0000BC0500200148FEF722
:10389000F5BE0000FC0500200C2000F0B7FFFEE79D
:1038A00003B401984100009850EAC12018BF0420D9
:1038B0004A0D18BF40F0010040F2FF72B2EB515FB9
:1038C00008BF40F00200012808BF052002B0704781
:1038D00070B52DED020B2DED0A8B82B00D98C40F43
:1038E00020F00045AE48854248D3AE48854219D302
:1038F0000C99C5F31300084309D09DED0C0B02B0E1
:10390000BDEC0A8B02B0BDE8704000F046BA002C56
:1039100014BF9FEDA50B9DED0C0B02B0BDEC0A8B07
:1039200002B070BD9FEDA20B53EC102B9DED0C0B64
:1039300051EC100BFCF7D8FF0AD2022000F068FA15
:1039400002B0BDEC0A8B02B0BDE8704000F030BAA6
:103950009FED990B53EC102B9DED0C0B51EC100BC4
:10396000FCF7AAFF0AD2022000F052FA02B0BDEC26
:103970000A8B02B0BDE8704000F02ABA90489FED73
:1039800092BBA8425CD29248854219D291487844B1
:1039900000EBC40090ED000B53EC102B9DED0C0BD5
:1039A00051EC100BFCF71FFD41EC1A0B8A487844D0
:1039B00000EBC40090ED009BC4F10100041B36E055
:1039C0009FED870B53EC102B9DED0C0B51EC100B66
:1039D000FCF70FFD41EC100B8348784400EBC4006A
:1039E00090ED001B51EC100B53EC112BFCF75AFC23
:1039F000FCF7FEFD0446FCF7DDFD41EC180B9FEDE6
:103A00007C0B53EC102BFCF7F4FC9DED0C1B53ECE2
:103A1000112BFCF7EBFC41EC1A0B9FED770B51ECF3
:103A2000180B53EC102BFCF7E4FC41EC190B51EC98
:103A30001A0B53EC192BFCF7D6FCCDE90C011BE05B
:103A40006F48854217D29FED700B53EC102B9DED04
:103A50000C0B51EC100BFCF725FC53EC1B2BFCF76B
:103A600043FF08D29DED0C0B53EC1B2B51EC100BBC
:103A7000FCF718FC6EE000249DED0C0B53EC102BB2
:103A800051EC100BFCF7B5FC41EC180B604805211C
:103A9000B0EE480AF0EE680A784400F002F953EC00
:103AA000182B51EC100BFCF7A4FC9DED0C1B53ECF8
:103AB000112BFCF79BFC41EC180B9FED570B5CB3F3
:103AC00053EC182B51EC100BFCF78DFC9DED0C0BFF
:103AD00041EC1C0B53EC182B51EC100BFCF789FC40
:103AE00053EC1C2BFCF7F7FC53EC192BFCF77EFC7A
:103AF00053EC1A2BFCF777FC53EC1B2BFCF776FCF2
:103B0000CDE900016FF47F70844226DB01EB0450A5
:103B100001909DED000B00E753EC102B51EC180BBE
:103B2000FCF761FC9DED0C0B41EC190B53EC182BD1
:103B300051EC100BFCF75DFC53EC192BFCF7CBFCA4
:103B40009DED0C1B53EC112BFCF74DFC53EC1B2B88
:103B5000FCF74CFC41EC100BDFE608464FF07A51C5
:103B600001EB04519FED2E0B084453EC102B0190F8
:103B70009DED000B51EC100BFCF73BFC0D4645ECAA
:103B8000100B044651EC100BFFF78AFE042808BF07
:103B900000F01EF945EC104BBFE6000000000000ED
:103BA000422E86400000F07F000000000000000070
:103BB000EF39FAFE422E864051302DD5104987C08C
:103BC000422ED63F00000000000000000000F03F41
:103BD000B2A2F03FAE3900009E39000000000000A4
:103BE000FE822B654715F73F5239000000000000A8
:103BF0000000E0FE422EE63F763C7935EF39EA3DA3
:103C00000000303E000000009C7500883CE4377ED8
:103C1000C438000000000000000000000000004068
:103C2000000000000000700100B52DED048BB0EE27
:103C3000409AF0EE609A83B051EC190BFCF7EBFD63
:103C400041EC180B18EE100A18EE901A8DED008B4F
:103C5000002818BF0120084320F00040C0F17F6019
:103C600000F1E040C00F14D019EE101A19EE900ABE
:103C70008DED009B002918BF0121084320F0004072
:103C8000C0F17F6000F1E040C00F04BF012000F0F0
:103C9000BFF8B0EE480A03B0F0EE680ABDEC048B42
:103CA00000BD70B504462DED028B4D1E00EBC50026
:103CB000B0EE408AF0EE608A90ED000B35F0060021
:103CC00017D053EC182B51EC100BFCF792FB41EC86
:103CD000100B6D1E04EBC50090ED001B51EC100B9A
:103CE00053EC112BFCF7DEFA41EC100B35F006001B
:103CF000E7D1022D36D0042D1CD0062D1CBFBDEC03
:103D0000028B70BD53EC182B51EC100BFCF771FBC0
:103D100094ED0A1B53EC112BFCF7C4FA53EC182B4F
:103D2000FCF767FB94ED081B53EC112BFCF7BAFA78
:103D300041EC100B53EC182B51EC100BFCF759FB1A
:103D400094ED061B53EC112BFCF7ACFA53EC182B3B
:103D5000FCF74FFB94ED040B53EC102BFCF7A2FA8D
:103D600041EC100B53EC182B51EC100BFCF741FB02
:103D700094ED021B53EC112BFCF794FA53EC182B27
:103D8000FCF737FB94ED001B53EC112BFCF78AFA80
:103D9000BDEC028B41EC100B70BD10B553EC102B39
:103DA00051EC100BFCF77EFA41EC100B10BD00003B
:103DB0009FED050B10B553EC102B51EC100BFCF7DD
:103DC00018FB41EC100B10BD00000000000000705B
:103DD0009FED050B10B553EC102B51EC100BFCF7BD
:103DE00008FB41EC100B10BD0000000000000010AB
:103DF00002E008C8121F08C1002AFAD170477047B4
:103E0000002001E001C1121F002AFBD17047000011
:103E100001490860704700000C02002010B586B010
:103E200040240194094802900020039001A9084809
:103E3000FDF7B6FA07480460002211461720FDF787
:103E400035FC1720FDF726FC06B010BD0000111050
:103E500000000240143C0140F0B41F4D2C69322C8C
:103E600033DA0022DFF874C002EB82030CEB830329
:103E70005B6843B1521C322AF6DB322A29D1F0BCEE
:103E8000042000F0C3BC02EB82034CF82300072897
:103E900014D2DFE800F004040B0B1013100091EDB6
:103EA000000A0CEB830080ED020A07E008880CEBA7
:103EB0008301C86002E00CEB830001610CEB83011D
:103EC00001204860601C2861D7E7F0BC032000F0A7
:103ED0009DBCF0BC70470000A8010020C4F5002084
:103EE00010B54FF400510448FDF760FB08B1002005
:103EF00010BD012010BD0000000802402DE9F8436C
:103F000007468846914600245A4E04EB44057069E2
:103F1000284400F0B1F870692844401C00F0ACF867
:103F200070692844801C00F0A7F8641CB4F5966FF3
:103F3000EBDBB9F1000F77D100254FF4966002F06A
:103F4000B3F800EB40047069015D00294DD12044B5
:103F50004178002949D18078002846D1404602F0B6
:103F6000A3F83844072870D2DFE800F004132231A8
:103F7000404F5F0001221146104602F017FA0090F0
:103F80007069BDF80010204401809DF80210817016
:103F900069E000221146012002F008FA00907069E1
:103FA000BDF80010204401809DF8021081705AE095
:103FB00000220121104602F0F9F900907069BDF865
:103FC0000010204401809DF8021081704BE0002118
:103FD0000122084602F0EAF900907069BDF800106D
:103FE000204401809DF8021081703CE001210022F4
:103FF000084602F0DBF900907069BDF8001020441B
:1040000001809DF8021081702DE0012211460020F0
:1040100002F0CCF900907069BDF8001020440180D6
:104020009DF8021081701EE021E00122002110465F
:1040300002F0BCF900907069BDF8001020440180C6
:104040009DF8021081700EE0FFE701221146104634
:1040500002F0ACF900907069BDF8001020440180B6
:104060009DF8021081706D1C042DFFF666AFBDE84F
:10407000F8830000E801002000B503461878FF2807
:1040800007D010F0010F07D0012101EB400018709C
:1040900000BDFE20187000BD0028FCD00421184689
:1040A00000F0BAFD187810F0010FF4D0401E18701F
:1040B00000BD00002DE9F04706462DED068BB0EE61
:1040C000409AB0EE60AAF0EE419A481E00EBD07024
:1040D0004FEA60089FED1B8A3446C8F100052F4661
:1040E00045451FDCDFF86090F0EE488A00EE105A7C
:1040F000F0EE690AB8EEC00A40EE090AB0EE4A0ACC
:1041000000F06AFE84ED000A10EE100A484501DA5C
:10411000C4ED008A94ED000A30EE088A241D6D1C5F
:104120004545E3DD474508DC96ED000AC0EE080A88
:10413000E6EC010A7F1C4745F6DDBDEC068BBDE8C9
:10414000F0870000000000000AD7233C70B5064647
:104150000024084D2046297801F016F8314600F079
:1041600049F808B1012070BD641C202CF2DB00204E
:1041700070BD0000D801002010B40023002A0DDD1E
:1041800010F803C0BCF13F0F05D0CC5CA44502D0B1
:1041900010BC002070475B1C9342F1DB10BC012077
:1041A0007047000010B584B004466946204600F010
:1041B00019FB6946204600F01DF840B102F036F9BF
:1041C0006846FFF7C3FF28B104B0012010BD04B05A
:1041D000002010BD06482246C1684B1C416800788B
:1041E00002F0BAFC02F022F904B0022010BD000077
:1041F000D801002000F56162002052F8203051F80B
:1042000020C0634501D000207047401C0428F4DB27
:10421000012070472DE9F843F14E7068002800D165
:1042200070707078EF49A1FB00214908A1EB810172
:10423000091806D001297BD0022900F0478100F03F
:1042400070B9AB214843400A48D0012854D0022815
:1042500060D003286ED0B42001F026FFC4B2B42091
:1042600001F022FFC5B2B42001F01EFFC0B2224609
:10427000294602F09BF800907069BDF8001001809B
:104280009DF8021081707069FF22831D114610464F
:1042900002F08CF80090BDF8001019809DF8020023
:1042A00098707069A0F803109A7842710388A0F89A
:1042B0000D3E837880F80F3EA0F80A1E80F80C2E81
:1042C000C188A0F8071E017A80F8091E7078401C8A
:1042D0007070082030610020BDE8F883002211468C
:1042E000B42002F063F800907069BDF800100180FE
:1042F0009DF802108170C6E70022B421104602F03A
:1043000055F800907069BDF8001001809DF802100A
:104310008170B8E70021B422084602F047F8009007
:104320007069BDF8001001809DF802108170AAE745
:104330000EE0FFE716229021B42002F037F800903B
:104340007069BDF8001001809DF8021081709AE735
:104350003069411C00FB01F2930903EB50153161F8
:10436000B3F5167F7DD20024012B40F2AF482CD04C
:10437000A3F10109706904EB44073844052100F0FA
:104380004BFC706905213844401C00F045FC706905
:1043900005213844801C00F03FFCA8EB040000EB32
:1043A000400770690521384400F036FC706905212A
:1043B0003844401C00F030FC706905213844801CF2
:1043C00000F02AFC641C4C45D4D3AB422FD8B3F583
:1043D000167F10DBFF221146104601F0E7FF009028
:1043E000716903EB43000844BDF8001001809DF89B
:1043F000021081700BE0706903EB43015A1E014407
:1044000002EB4202104402880A8080788870A8EB90
:10441000030000EB4001706903EB430201441044C8
:1044200002880A80807888705B1CAB42CFD9A81CB8
:1044300000EB40047069FF2223181146104601F07A
:10444000B5FF0090BDF8000018809DF8021099702B
:10445000691C726901EB41010A44108098789070E0
:1044600000E018E040F2AE40401B00EB40027069F3
:1044700002440844018811808078907040F2AD4079
:10448000401B00EB400170690144204402880A800F
:104490008078887017E00023FF221146104601F053
:1044A00085FF0090716903EB43000844BDF80010DC
:1044B00001809DF8021081705B1CB3F5966FEBDBF9
:1044C0007078401C70700020BDE8F88371690A782C
:1044D0001AB94A780AB9897831B300237078AB21C8
:1044E00010FB01F0400A2AD001283CD002284ED00F
:1044F000032860D0706903EB43042044042100F0DA
:104500008BFB706904212044401C00F085FB70691E
:1045100004212044801C00F07FFB5B1CB3F5966FE8
:10452000DCDB0020BDE8F883401CC0B270700F28AF
:1045300002D00020BDE8F8830120BDE8F88370694F
:1045400003EB43042044032100F066FB706904215F
:104550002044401C00F060FB706902212044801C54
:1045600000F05AFBD9E7706903EB430420440421AF
:1045700000F052FB706903212044401C00F04CFB0A
:10458000706902212044801C00F046FBC5E7706979
:1045900003EB43042044042100F03EFB7069042136
:1045A0002044401C00F038FB706903212044801C2B
:1045B00000F032FBB1E7706903EB430420440321B0
:1045C00000F02AFB706902212044401C00F024FB0B
:1045D000706904212044801C00F01EFB9DE7000050
:1045E000E8010020ABAAAAAA2DE9F84F8246DFF81D
:1045F0005C8100220921D8F81400C31C00F0A8F83F
:10460000D8F814000022031D0921401C00F0A0F876
:10461000D8F814000022431D0921801C00F098F8EE
:10462000012440F2AF49601C00EB4005D8F814109B
:10463000601E00EB400604EB44076B1872187818F4
:10464000092100F085F8D8F8140029184B1C3118FE
:104650004A1C3844401C092100F07AF8D8F81400AC
:1046600029188B1C31188A1C3844801C092100F041
:104670006FF8641C4C45D6DBD8F81400002300F614
:104680000A620921D01C00F063F8D8F81400002356
:1046900000F60B620921D01C00F05AF8D8F814007B
:1046A000002300F60C620921D01C00F051F8BAF189
:1046B000000F48D1002501264FF4966001F0F4FC6C
:1046C0000446072001F0F0FC072839D2DFE800F0AB
:1046D00004040C0C15153000D8F8141004EB440039
:1046E0000A5C22BB0E542BE0D8F8141004EB4400F3
:1046F00008444178D9B9467022E0D8F8140004EB98
:104700004403C15C99B91844417881B9807870B983
:1047100001221146104601F049FE0090D8F814001D
:10472000BDF80010184401809DF80210817007E068
:10473000D8F8141004EB44000844817801B986705D
:104740006D1C012DB8DBBDE8F88F0000E8010020EA
:1047500070B5064614461D4630781F280CD1481CFB
:1047600001F0A2FC40B1012114B1207800B9217000
:1047700015B1287800B929703046BDE87040FFF7C0
:104780007BBC000070B505460E460D4C2278032A0E
:1047900001D0042A0CD100F057FDD4ED030A0948DA
:1047A00030EE600A10EE102A824201DD01202070F6
:1047B00001F0E6FB31462846BDE8704000F0F6BC4B
:1047C000A80100200000A0400020054A002100EBC5
:1047D000800302EB83035960401C3228F7DB7047EB
:1047E000C4F5002070B506460D460024C4EB441005
:1047F000C0EB042006EB80004FF4617100F052F82A
:1048000045F82400641C042CF0DB70BD2DE9F04158
:1048100005460026DFF88880012701222021404636
:10482000FCF7CFFE282001F0DBFA002220214046D1
:10483000FCF7C7FE142001F0D3FA012220214046E4
:10484000FCF7BFFE282001F0CBFA002220214046D1
:10485000FCF7B7FE4FF4C87001F0C2FA0024C4F1AF
:10486000070007FA00F0284204D001222021404628
:10487000FCF7A7FE642001F0B3FA00222021404695
:10488000FCF79FFE4FF4C87001F0AAFA641C082CD4
:10489000E5DB761C142EC0DBBDE8F04101F0DABA8E
:1048A00000000240F0B507464FF0FF33CD00002472
:1048B000002D0EDD084E2146384600F04DFCB0EBD1
:1048C000D37F02D086EA430300E05B00641CAC4265
:1048D000F1DB1846F0BD0000DB114C1070B52DED7A
:1048E000028B0125364C2178002912D1002204F1D7
:1048F000480C5CF82130C3EB031302EB83024CF845
:104900002120491C3429F4D362614FF0FF31E1606A
:10491000257030B184ED040A00206070BDEC028B7C
:1049200070BDD4ED040A70EE600AFCEEE00A10EEF1
:10493000900AB0F5167F01D9012000E000206178CF
:104940000843EBD0BDEEC00A616910EE100AB0FB5F
:10495000F1F201FB120000F0E7F91A49085C60630C
:10496000E16888421ED016289FED170A18D2062843
:104970000ED00A280CD00B280DD09FED148AB0EE73
:10498000480A01F0CDFDB0EE480A01F077FD09E0DC
:1049900001F0C6FD06E09FED0E0A01F0C1FD01E049
:1049A00001F0BEFD616BE068814204D0072801D0B0
:1049B00007206063A570606BE060BDEC028B70BD8A
:1049C000000000201C720008CDCCCC3C0000000090
:1049D000CDCC4C3D00B585B00848016821F04001C0
:1049E000016007494020086000900020019002907B
:1049F00069460448FCF7D4FC05B000BD003C01400A
:104A0000143C01400000024000224FF400410148E4
:104A1000FCF7D7BD0000024070B50D46184C0023CE
:104A20002360184A1360014641F269131648FCF7E7
:104A30008BFB41F26913224629461448FCF784FB9C
:104A4000134C2068C16841F40071C1602068C168DE
:104A500041F40061C1600F4D012200212846FEF79C
:104A60009FFB012208212846FEF79AFB2068416C33
:104A700041F400414164016841F00101016070BDF1
:104A80001408024014040240640500200C050020B4
:104A9000D00400200004014010B51B4C0022114638
:104AA0002046FEF77DFB002208212046FEF778FB1A
:104AB000164A1068036A41F211110B4240F2444356
:104AC0000AD1D0F820C01CEA030F05D1D0F844C0A9
:104AD0002CF4004CC0F844C0D0F820C01CEA010FF0
:104AE00006D1016A194203D1016821F00101016078
:104AF0001068C16821F40071C1601068C16821F4B8
:104B00000061C16010BD000000040140D00400201D
:104B100010B50E490E4800F059FD0C490C48FFF73E
:104B20007BFF0420FCF758FB142200210948FCF706
:104B300055FA142200210848FCF750FAFFF7ACFFA1
:104B4000BDE810400420FCF747BB00005E61002078
:104B50008C3E0020640500200C05002010B50A489A
:104B60000068016821F001010160084800680168DF
:104B700021F0010101600448FCF7C8F8BDE81040CD
:104B80000248FCF7C3B80000640500200C050020B3
:104B900010B5142200210C48FCF720FA20B1BDE822
:104BA00010400820FFF732BE142200210748FCF70E
:104BB00015FA20B1BDE810400920FFF727BEBDE877
:104BC0001040FFF769BF0000640500200C050020BD
:104BD0000122D1030148FCF7F4BC000000000240B0
:104BE00000224FF480710148FCF7EBBC000002404A
:104BF00000B587B0002102910121039105910221A6
:104C000006910490FCF794FB01A902A8FCF7F0FAC6
:104C1000FCF744FB07B000BD0278002A05D022FA59
:104C200001F101B90121511A017070472DE9F041DC
:104C300088B014461D46B0EE601AF0EE400AB7EE9A
:104C4000000A052103A8FFF735FA00230027DFED4E
:104C5000350A0DF10C084FF0000CC7EB0716CDED2F
:104C6000020ACDED010ACDED000A6FF001010CEB57
:104C70000100002801DA3C3002E03C2800DB3C382F
:104C800000EB860000EB40008A1C08EB82029DEDE1
:104C9000001A92ED000A421C205C01EE900AF8EE28
:104CA000611A00EE211A8DED001A501CA25C9DEDD8
:104CB000011A01EE902AF8EE611A00EE211A8DED2C
:104CC000011A205C9DED021A01EE900AF8EE611ABD
:104CD00000EE211A8DED021A491C0229C7DD9DED57
:104CE000000ABCEEC00A10EE100AE8549DED010A5D
:104CF000E818BCEEC00A10EE101A41709DED020AD1
:104D0000BCEEC00A10EE101A8170DB1C0CF1010C15
:104D1000BCF13C0FA3DB7F1C142F9CDB08B0BDE86B
:104D2000F08100000000000001460020044A52F813
:104D300020308B4203D8401C3428F8D30A20704717
:104D4000480000202DE9F047824689464FF0FF35A4
:104D500000262F46A84600245146204600F01CFAA3
:104D6000B0F1FF3F07D0B04200D90646B84206D2A4
:104D7000A046074603E0B5F1FF3F00D12546641C7D
:104D8000202CE9DBB5F1FF3F00D1454617601E60DE
:104D9000C9F80050BDE8F08770B506460D461446C8
:104DA000FCF7C6FA002C0ADD0023314602202A68EF
:104DB000FCF77EFA2D1D361D241F002CF4DCBDE807
:104DC0007040FCF76BBA000002480068406880B28F
:104DD00070470000BC05002010B52DED048BB0EE2F
:104DE000409AB1EE600A60EE200AB0EE000A29EEA9
:104DF000000A20EE091A80EE810A10EE100AFBF775
:104E000016FC41EC100BFEF763FDB0EE408AF0EEAD
:104E1000608A19EE100AFBF70AFC41EC190B9FEDB2
:104E2000100BFEF701FF53EC192B51EC100BFBF7A5
:104E3000E0FA41EC100B53EC102B9FED0B0B51ECF7
:104E4000100BFBF748FB53EC182BFBF7D2FAFBF7E0
:104E500001FCBDEC048B00EE100A10BD0000000048
:104E600000000060FB211940000000000000F03F3E
:104E700010B54FF46161FBF7ECF9002010BD0000A4
:104E80002DE9F05F06462DED028BB0EE408A8A4692
:104E9000644F00244FF0010B387800281FD097EDA5
:104EA000010A38EE400A10EE100AB0F1804F16DC0D
:104EB000D7ED020AF5EEC00AF1EE10FA06D078EE50
:104EC000600A594910EE900A884208DCD7ED030ABF
:104ED000564978EE600A10EE900A884219DD7C701F
:104EE00087F802B0B3EE040A28EE000ABCEEC00A4E
:104EF00010EE100AFBF78CF901F0B8F887F800B053
:104F00009FED4B0A87ED020A87ED038A87ED018A40
:104F100011E010EE100A4749884204DABDEC028B1A
:104F20000120BDE8F09F7878C0F101007870B87872
:104F3000C0F10100B8704FF00009DFF8FC800024D8
:104F4000C9EB091522464946787800F0C3F879780C
:104F5000C1EB011101EB810108EB011101EB8501AE
:104F6000095D41B3012940D00020FFF74FFC04EB5D
:104F7000850000EB4001B878C0EB001000EB80002A
:104F800008EB001000EB8500005D00FB0AF04A1CF6
:104F90007054511CB0547054641C3C2CD2DB09F189
:104FA0000109B9F1140FCADB87ED018A0120BDECBC
:104FB000028BBDE8F09F03280BD0B8780021C0EB2E
:104FC000001000EB800008EB001000EB850001559D
:104FD000CDE7B878C0EB001000EB800008EB0010C4
:104FE00000EB850000F804B0C1E702280DD00328CB
:104FF0000BD0B8780021C0EB001000EB800008EB6C
:10500000001000EB85000155B1E7B878C0EB001047
:1050100000EB800008EB001000EB850000F804B006
:10502000A5E700003C010020000020410000704284
:10503000000000009A99993E34CB002078B50646CE
:105040000C4600258DF800508DF801408DF8025077
:105050006A462946304600F0C5FF14218DF80050FD
:105060008DF801408DF802506A46304600F0BAFFD4
:1050700028218DF800508DF801408DF802506A46C5
:10508000304600F0AFFF002078BD00220B7800F81A
:10509000013B4B7800F8013B8B7800F8013B521C38
:1050A000B2F5966FF2D30020704710B50A464FF460
:1050B0006161FBF7C7F8002010BD08B58DF801103D
:1050C0008DF8001089088DF802106946FFF7DDFFA2
:1050D000002008BDF0B4002931D04D1E132931D075
:1050E0004C1C72B3531E3B2A30D002F1010CC0EBB2
:1050F000001000EB80061748C5EB051500EB061005
:1051000000EB8505C1EB0111AF5C00EB8101EE5CAA
:10511000C4EB04143E44CF5C15F80C5000EB840043
:105120003D4411F80C103544C35C2944825C10F8EE
:105130000C001944F0BC11440844C0B27047132558
:10514000CCE701E00024CCE73B23CCE74FF0000C98
:10515000CDE7000034CB002000EBE10001F00701B7
:105160000078012202FA01F1084201D001207047C3
:105170000020704703480068406841F21021081A77
:1051800070470000D4C90020490401EB003000F151
:10519000006000F580207047490401EB00300249AF
:1051A0000844006870470000200E040870B584466B
:1051B0000846234E316900290DD00022214D02EB13
:1051C000820305EB83035968012906D0521C322A59
:1051D000F5DB002070BD002070BD02EB820455F8A5
:1051E0002410CCF80010072920D2DFE801F00404D5
:1051F0000B0B101F180005EB840191ED020A80EDE6
:10520000000A13E005EB8401C96801600EE005EBBC
:1052100084014FF461620969FBF702F806E005EBCF
:1052200084014FF462620969FAF7FAFF05EB840121
:10523000002048603069401E3061012070BD0000D0
:10524000A8010020C4F500200C48016821F00101EC
:105250000160416A89B20A4A92ED000A026842F08E
:105260000102026000EE901AB8EE400A9FED051AA6
:10527000F8EE600A00EE810A70470000001000405E
:105280004C01002017B7D13870B50646124C0025E6
:1052900025703046FAF7E8FF25543046FAF7E4FF68
:1052A00082B241F2883321460C48FDF743FB40B1FE
:1052B00001280DD002280BD0032809D00220FFF7C7
:1052C000A5FA05493046FAF7D6FF18B1012070BD9E
:1052D000032070BD002070BD94D40020BC050020C8
:1052E00000F0ECFD01F0CAFAFBF7F8FC10B5FFF78F
:1052F00077FC0B4C00224FF400612046FCF761F96B
:10530000012202212046FCF75CF9FFF761FC4FF413
:105310007A7001F0A9FABDE8104001F039B8000038
:105320000000024010B5FFF75BFC0B4C00224FF46D
:1053300000612046FCF745F9002202212046FCF7D7
:1053400040F9FFF745FC4FF47A7001F08DFABDE8A3
:10535000104001F01DB80000000002402DE9F841A6
:105360000023744F744DA0264FF496680024B3F5C3
:10537000966F2ED2604200EB800006EB800000FBAF
:1053800004F101EB8101890087FB01218A11A2EB65
:10539000E171CAB204EB84018906090EC0B201F0C2
:1053A00005F80090686803EB500000F59660B0FBCC
:1053B000F8F108FB1100696900EB40000844BDF8F2
:1053C000001001809DF8021081705B1C641C082C89
:1053D000CDDB0024B3F5966F2ED2604200EB800047
:1053E00006EB800000FB04F101EB8101890087FBE3
:1053F00001218A11A2EBE171CAB2C1B204EB8400AF
:105400008006000E00F0D2FF0090686803EB5000A9
:1054100000F59660B0FBF8F108FB1100696900EB3C
:1054200040000844BDF8001001809DF80210817012
:105430005B1C641C082CCDDBB3F5966F96D340F251
:10544000C2410020002601226B680344B3FBF1FC3B
:1054500001FB1C338446401C8C4569D2B3F5966F22
:1054600017D2D5F814C003EB43031CF80340D44013
:105470000CF803409C449CF80140D4408CF8014057
:10548000D5F814C0634493F802C02CFA02FC83F8E8
:1054900002C0521C082AD7DB00226B680344B3FB0E
:1054A000F1FC01FB1C338446401C8C4540D2B3F513
:1054B000966F0CD2D5F814C003EB43030CF80360CD
:1054C0009C448CF80160D5F814C063449E70521C53
:1054D0000A2AE2DB00226B680344B3FBF1FC01FB08
:1054E0001C338446401C8C4522D2B3F5966F19D2EA
:1054F000D5F814C003EB4303C2F107041CF8037092
:10550000E7400CF803709C449CF80170E7408CF86D
:105510000170D5F814C0634493F802C02CFA04FC5F
:1055200083F802C0521C072AD5DB401D88428AD36B
:10553000BDE8F88167666666E801002070B504463C
:105540000D46162C39D2DFE804F00B0D0D0D0D0DB4
:1055500012171B20252A2F2F2F2F2F2F2F2F2F34BD
:1055600000202AE0E1B2284601F01CFC25E01146AB
:105570002846FFF763FD20E02846FFF779FC1CE092
:1055800011462846FFF791FD17E011462846FFF720
:1055900094FD12E011462846FFF750FD0DE011463C
:1055A0002846FFF76DFC08E0E1B2284601F0FAFB5F
:1055B00003E0284600F072F90120162C05D3A4F16F
:1055C0001601284600F0C4FE002070BD00224FF6F0
:1055D000FF7C002320F802CB21F802CB20F8023B0D
:1055E00021F8023B20F8023B21F8023B521CB2F5A5
:1055F000B46FEFD3002220F8023B21F8023B521C8B
:10560000892AF8D3704700002DE9F041124D002699
:105610006E700024114F05F1140858F82400FAF7B1
:1056200023FE47F824006978884200DD6870641C16
:10563000072CF2DB6878202802D90720FFF7E6F86C
:1056400000206978002904DD054A1654401C884270
:10565000FBDB2E61BDE8F081A8010020ACF9002041
:10566000C8F900202DE9F04707460C461546AC4224
:1056700002D10020BDE8F087DFF8348198F80010EF
:10568000032909D0042907D001296CD00520FFF790
:10569000BDF80020BDE8F087A5420CD241F21022EF
:1056A00021463846FFF7DEFF18B1284480B2BDE836
:1056B000F0870024DBE7281B1FFA80F93C4A3D48AD
:1056C000A5EB040C12893B191FFA8CFC104494447E
:1056D000032902D1BCF5616F04D2042936D1BCF58F
:1056E000626F33D3032902D0042904D006E0C2F547
:1056F00061618EB202E0C2F562618EB2A9EB060171
:105700001FFA81F932461946FAF78AFDB8F80800FF
:105710003044A8F8080098F8000003280ED0254966
:105720000620FEF799FB012088F80000B9F1000F70
:1057300009D0A01981B22A46384695E71D490420B0
:10574000FEF78AFBEFE70020BDE8F08700244A4619
:105750001946FAF765FDB8F808004844A8F80800AB
:105760002046BDE8F087A5420CD241F21022214626
:105770003846FFF777FF18B1284480B2BDE8F087BC
:10578000002474E7AC420BDA385D00F015F898F8A5
:105790000010032907D0042905D0641CAC42F3DBB8
:1057A0000020BDE8F087601C81B22A4638465BE7DE
:1057B000A8010020A4E700202DE9F04F83B00021CC
:1057C000324FDFF8CC807A78521E002A07DD08EBD2
:1057D00001035B7808F80130491C9142F7DB08F8B7
:1057E00001000024DFF8AC9000264FF0040A59F8BD
:1057F00024207878801A80B208EB000526482946D4
:1058000050F82400FEF7B8FC20B3072C37D2DFE8AD
:1058100004F00404101022322A00EE7405F10C008A
:1058200000F052FD8DED020A02A92046FEF714FB9E
:1058300025E005F10C0000F032FD834605F10E0075
:1058400000F02DFD014641EA0B40019001A92046E0
:10585000FEF702FB13E003203870FFF7F5FC87ED3D
:10586000030A3E810BE087F800A0FFF7EDFC87ED0F
:10587000030A3E8103E000212046FEF7EDFA641C96
:10588000072CB4DB03B0BDE8F08F0000A8010020B6
:10589000C8F90020ACF90020BC01002038B5644CE8
:1058A00060616068002814D1002300221146104670
:1058B00000F07CFD0090616903EB43000844BDF8F3
:1058C000001001809DF8021081705B1CB3F5966F8B
:1058D000EBDB584D32202860207808B1012811D127
:1058E00055496068A1FB00218908A1EB810110EBFB
:1058F000410004D147F2305000F0D6FBA060A06810
:10590000FAF786FC21784FF4FA60072979D2DFE8AC
:1059100001F0041223294044720040F6B830E060E0
:10592000606840F67231884201D9012000E0002011
:1059300000F0CEFF65E04FF47A60E0606068B0F59B
:10594000756F01D9012100E0002118B1002000F09D
:10595000B7FB56E00120FAE74FF44870E06000F032
:1059600049FE4EE0E06035496068A1FB00218909ED
:105970006FF01802514300EBC101822903D840F2B5
:105980006C71884201D9012000E00020FEF72CFE56
:1059900037E0E060FFF7E2FC33E04FF49660E06050
:1059A0001E2028606068B0F5C87F05D20022012162
:1059B0001046FEF7A3FA24E040F28A21884205D27D
:1059C000002202211046FEF799FA1AE0B0F5617F35
:1059D00005D2002202210120FEF790FA11E040F2E8
:1059E0004C41884201D9012200E000220621012019
:1059F000FEF784FA05E0FEF70DFC10B96068801C24
:105A0000E0606068401C6060E16888420ED300205E
:105A1000606020780A4B401CC0B21A460021E0FBAF
:105A200003214908A1EBC1010844207038BD0000E2
:105A3000E80100201C000020ABAAAAAA1F85EB5198
:105A400049922449FEF7E2BE2DED068B82B0DFF8C5
:105A500034B3CB48CBF80000CB48CBF804000BF1B3
:105A60000806CA483060CA487060CA4C4FF0000A45
:105A7000C4F800A0C84FC7F800A0C84DC5F814A0CE
:105A8000FBF7B4FDFDF7A4FAFDF7D2F8FDF78AF8AD
:105A9000FDF764F9FDF780F9FDF7A4F9FDF7BEF90C
:105AA000FDF7D6F9FDF71AFAFDF740FAC4F800A0A1
:105AB000C7F800A0C5F814A0FEF7A6FFFFF790F8FE
:105AC000B748816841F002018160816841F01001AE
:105AD0008160816841F020018160B248FCF716FCCA
:105AE000B148FCF713FC00F023FA10B91020FFF7BF
:105AF000A9FFAE48802707704021417081700146A0
:105B0000AB48FFF7C2FA022211463620FBF7CEFD62
:105B1000A84CC4F810A03620FBF7BCFDE06840F0AC
:105B20000100E06000F03CFC00F0D6FCFEF7D8F984
:105B300008B100F00DFF00F0E1FC00F029FD10B904
:105B40000D20FEF763FE00F00BFD00F06FFC9FEDF3
:105B50009A8AB0EE480A00F0E3FCB0EE480A00F082
:105B60008DFC4FF0010800243168DBF80000FFF7DE
:105B70002DFD7168DBF80400FFF728FD8F484FF01A
:105B80000109C0F8349080F80290C7708C4DB7EED0
:105B9000009ADFED8C9ADFF830B207469FED8C8BD0
:105BA00000266420F86186496846FEF7EBFD002870
:105BB0003FD001260098072835D2DFE800F0040D19
:105BC000163023611F0095ED000A00F057FC2021DC
:105BD0007248FBF7F2FC26E095ED000A00F0A0FC0D
:105BE00020216E48FBF7E9FC1DE02868786387F800
:105BF000029020216948FBF7E0FC14E07048FEF7B2
:105C0000D1FA80B14FF461626D496948FAF708FB37
:105C1000C7F834A020216148FBF7CFFC03E02878C7
:105C2000F87087F8029066496846FEF7ABFD0028D9
:105C3000BFD101A800F0CAFD87ED0A0A30469DEDEC
:105C4000010AFEF74BFE97ED0A0AFDEEC00A10EEC0
:105C5000900A386300EE900AF8EEE00A30EE600A2F
:105C600087ED0B0A10EE101AB1F17C5F16DD30EEF5
:105C7000490A87ED0B0A401C38633C280CD00DE024
:105C800040F6B830DBF800108142FBD3FEF780FF0E
:105C9000FEF73EFF00F0DEF8C7F830A0B87838B164
:105CA000FA789DED010A4249786BFFF747FCB8701E
:105CB0003F49FA7801F5616001F064FA28B93C497E
:105CC000FA7801F5616001F04AFA97ED0B0A424B50
:105CD0001421F1EE400AA3F561623C20B0EE690A9E
:105CE000FEF7A4FF274850F824103962083050F816
:105CF00024207A6297F83030374800F08DFFB8F1F1
:105D0000000F04D1FEF744FFDBF80000F8803349B0
:105D10000198884201DD00F09DF8F869FAF74AFC25
:105D200041EC100B51EC180B53EC102BFAF7D3FB92
:105D3000FAF75EFCDBF800108142FBD3796A386A1F
:105D4000FEF76AFEDBF8000080B2B880CBF800A056
:105D5000FAF741FC41EC100BB0EE48AAF0EE68AA4D
:105D600053EC102B51EC1A0BFAF7B5FBFAF772FC57
:105D7000B8614FF00008C4F1010411E70000000011
:105D80008C3E002038000020308400205E6100201E
:105D900002A7002014080240140402400000024040
:105DA000002004E058040020940400200800002093
:105DB0003C06002000100040000000000000002011
:105DC0006C3000203333333F2414004000000000C7
:105DD0000000000080842E415C22002000A00C47BF
:105DE00010B504460023002C06DD4FF47A7000F055
:105DF0003BFD5B1CA342F8DB10BD000070B5134CEB
:105E000020680168124D11F0200F0BD04068C1B21C
:105E10002868026812F0800F01D0416002E00F2074
:105E2000FEF7F4FC2868016811F0200F07D04068E5
:105E3000C1B22068026812F0800F01D0416070BDCD
:105E4000BDE870400E20FEF7E1BC0000BC0500205C
:105E5000FC05002082B000F04DF8144C6420FFF7E0
:105E6000BFFF134901A8FEF78DFC40B1019805283A
:105E70000ED00F4901A8FEF785FC0028F6D1FFF7E8
:105E8000E3F910EE100AA042E8DDFFF729FAE5E792
:105E9000BFF34F8F07480168074A01F4E0611143DF
:105EA0000160BFF34F8F00BFFDE7000000207D4879
:105EB0006C3000200CED00E00400FA0510B5FEF790
:105EC00089FD09490020086008490860084C8021C4
:105ED000616100222046FBF774FB20460022BDE8EA
:105EE00010402021FBF76DBB14080240140402404F
:105EF0000000024010B5FEF76DFD0A490020086061
:105F000009490860094C48F2801161610022802132
:105F10002046FBF756FB20460022BDE8104020211A
:105F2000FBF74FBB1408024014040240000002407B
:105F300070B5124D012280212846FBF742FB002458
:105F40006420FFF74DFF40212846FBF72FFB58B197
:105F5000641C322CF4DB322C09DA01222021284681
:105F6000FBF72FFB012070BDFDF758FFF3E7002280
:105F700080212846FBF725FB002070BD0000024071
:105F80002DE9F041FFF7F6F80446144EB088A04220
:105F900022D041F21027A2B2B1881148FFF762FB6C
:105FA0000546B088844203DA391A214489B201E0F7
:105FB000211A89B2491B084480B2B080B84203D389
:105FC000A0F590501038B080B088B84202D30620B7
:105FD000FEF71CFC002DDED1BDE8F081A8010020F9
:105FE00094D500202DE9F0010027DFF87C8007EB35
:105FF00087035B00C7EB071C01EB8C0C0CEB4C041C
:106000004FF0000CBCF10A0F01DBA3F1010315787E
:1060100018F8036015FB06F54FEA152504F1010693
:106020000555547818F8035014FB05F44FEA14246E
:1060300006F101058455947818F8036014FB06F402
:106040004FEA142605F10104465501DA03F1010374
:106050000CF1010CBCF1140FD4DB7F1C142FC6DB38
:10606000BDE8F00170470000507200082DE9F041D2
:106070000025DFF830806FF040470024C5EB0510A5
:1060800008EB8006FAF7BAF8B84201DB012000E01D
:1060900000203055641C3C2CF4DB6D1C142DECDB13
:1060A000BDE8F08134CB002010B50446FAF7A6F81D
:1060B00000146043C11700EB5140C01310BD000035
:1060C0002DE9F84380460D460224654FB8F1000FD4
:1060D0007DD0B8F1010F79D0B420FFF7E5FF00F0D3
:1060E000FF09B420FFF7E0FFC6B2B420FFF7DCFFE2
:1060F000C0B24A46314600F059F90090796904EB84
:1061000044000844BDF8001001809DF80210817021
:10611000012C19DB7B6904EB4401C818595C8278B7
:1061200040788B08800801469208184600F03EF936
:106130000090601E796900EB40000844BDF8001033
:1061400001809DF802108170022C18DB786904EB45
:1061500044010B18405C9A785B78D208DB08C008D1
:10616000194600F023F90090A01E796900EB400069
:106170000844BDF8001001809DF802108170601C79
:10618000B0F5966F0BDA00EB40017869621E0144AE
:1061900002EB4202104402880A8080788870A01CBA
:1061A000B0F5966F0BDA00EB40017869A21E01444E
:1061B00002EB4202104402880A8080788870E41D55
:1061C000B4F5966F82DBBDE8F88300E022E00DB104
:1061D000012300E00323786904EB440630440322E2
:1061E000B42100F03FF80DB1012300E003237869EA
:1061F00003223044401CB42100F034F80DB10123D7
:1062000000E00323786903223044801CB42100F0AD
:1062100029F87DE714F0010F10D000221146B420B8
:1062200000F0C4F80090796904EB44000844BDF81C
:10623000001001809DF80210817069E70022B421EE
:10624000104600F0B3F80090796904EB440008446C
:10625000BDF8001001809DF80210817058E7000021
:10626000E801002070B504460E4615461846FFF7B3
:106270001BFFC0B240B1012805D12078711B8842B4
:106280000BDC2844207070BD2078A84202D3401B4C
:10629000207070BD0020207070BD267070BD017828
:1062A000412902D33739C9B201E03039C9B2407847
:1062B000412802D33738C0B201E03038C0B200EB19
:1062C0000110C0B27047000001782D2935D001219E
:1062D0004278303A00EE102AB8EEC00AC2789FED3C
:1062E000181A303A00EE902AF8EEE00A00EE810A21
:1062F00002799FED141A303A00EE902AF8EEE00A87
:1063000000EE810A42799FED101A303A00EE902A91
:10631000F8EEE00A00EE810A80799FED0C1A303821
:1063200000EE900AF8EEE00A00EE810A00EE901A04
:10633000F8EEE00A20EE200A70474FF0FF31C7E781
:10634000CDCCCC3D0AD7233C6F12833A17B7D13856
:1063500010B504460846202804DA0C49421CCB68D4
:106360009A4207D92046BDE8104040224FF46161AF
:10637000F9F768BF0978FEF707FF01462046BDE838
:1063800010404FF46162F9F74BBF0000D8010020C4
:10639000012211020148FBF714B90000000002407D
:1063A00001490120087070475C01002081B08DF820
:1063B00000008DF80110BDF8000040EA024001B075
:1063C0007047000070B50546154E56F82500F9F7E0
:1063D0004BFF044656F825101248F9F75AFF1148AA
:1063E0000D21015520440A21417000218170A01C1B
:1063F00082B24FF47A730B490B48FCF75DFB60B136
:10640000012808D0022806D0032804D00220FEF775
:10641000FDF9012070BD002070BD012070BD00009D
:106420006801002094D40020BC05002000B586B08F
:10643000002001AB03AA05A9FEF784FC01206B46EE
:1064400002AA04A9FEF77EFC019900980A4A884234
:1064500008D9012111700499516002999160D060AE
:1064600006B000BD00201070059850600398906041
:10647000D16006B000BD0000D801002000B510EECC
:10648000100ADFED120A10F1814F02D3B0EE600A5C
:1064900010E010EE100AB0F17E5F02DBB0EE600A91
:1064A00008E0B5EEC00AF1EE10FA03D2F7EE000AEA
:1064B00030EE200ADFED060A064B20EE200A83EDBF
:1064C000020AFEF7C1FE83ED030A00BD00000000D2
:1064D000000070424C01002000B585B04FF4005020
:1064E0000090002001900290039069460248FAF75C
:1064F00057FF05B000BD00000008024000B585B0A0
:106500004FF400500090012001900021029103906F
:1065100069460248FAF744FF05B000BD0008024092
:1065200008B5F0EE401A684600F050F911EE900AF6
:10653000B0F17E5F01DDF7EE001A11EE900A10F166
:10654000814F01D9FFEE001A9FED030A034821EEA7
:10655000800A80ED010A08BD000070424C01002055
:1065600010B5FEF731F9FFF74FF8064900204880D3
:106570008880C880BDE8104041F2102202490348DB
:10658000FCF74EBAA801002094D50020BC050020DD
:1065900070B5FEF7ABFE4FF4FA60FFF721FCC8239D
:1065A000062210491048FCF787FAC820FFF718FCAC
:1065B000FEF70AFC00240D4D2046FFF703FF30B123
:1065C00055F82400FEF760FE18B1002070BD0020D1
:1065D00070BD641C082CEFDB054902200870012007
:1065E00070BD000061010020BC0500208801002072
:1065F000600100202DE9F043714C60680A2832D315
:106600004FF4966500236F4E6F4F984660680A38C6
:10661000A6FB002109094A4202EB820200EB82003C
:10662000401CC9B21944B1FBF5F205FB1211B1F5DA
:10663000966F15D213F0030F17D001EB4109606973
:1066400003214844FEF7E8FA606903214844401CEE
:10665000FEF7E2FA606903214844801CFEF7DCFA89
:106660005B1CAB42D2D3BDE8F083DA1703EB927226
:10667000921087FB029C4FEA6C09A9EBEC7CCCF1F1
:10668000000C0CEB8C0C6244052AE9D2DFE802F026
:10669000031E3C587300C82242434CF6CD4C02FB0B
:1066A0000CF24FEA125C626901EB410102F801C091
:1066B00000EB8000400040F6CD4C00FB0CF00A449B
:1066C000000C5070626911448870C9E700EB8002C9
:1066D000520040F6CD4C02FB0CF2D4F814C001EB92
:1066E0004101120C0CF801204FF0C80900FB09F021
:1066F0004CF6CD4900FB09F08C44000D8CF80100EC
:10670000606908448270ABE7C82242434CF6CD4C26
:1067100002FB0CF24FEA125C626901EB410102F8E4
:1067200001C0C0EB0010C00046F2676C00FB0CF02B
:106730000A44C00C50706069084480F802808FE7FA
:1067400000EB8002520040F6CD4C02FB0CF2D4F874
:1067500014C001EB4101120C0CF801208C448CF8A0
:106760000120C82250434CF6CD4250436269000DCF
:106770001144887074E7C82242434CF6CD4C02FBAA
:106780000CF24FEA125C626901EB410102F801C0B0
:106790004FEA801C40F6CD490CFB09FC0A444FEA45
:1067A0001C4C82F801C000EB001202EBC0104CF64A
:1067B000CD4250436269000D1144887050E70000DB
:1067C000E8010020CDCCCCCC6766666610B50446E7
:1067D000FEF73AFD84ED000A2049D1ED010AF5EEFD
:1067E000C00AF1EE10FA04D181ED030A91ED020A1C
:1067F00010BD91ED031A30EE411A91ED020A01EE3F
:10680000200A81ED020A10EE100A154BDFED150A81
:10681000984209DB91ED020A30EE600A81ED020A2E
:1068200010EE102A9A42F5DA91ED020AB5EEC00A8E
:10683000F1EE10FA0AD291ED020A30EE200A81ED53
:10684000020AB5EEC00AF1EE10FAF4D394ED000A94
:1068500081ED030A91ED020A10BD00004C010020F9
:106860000000704200007042034900220A600A687A
:106870008242FCD370470000241400402DE9F0410F
:106880002DED028BFCF76AFBFEF7DEFCB0EE408AD2
:106890000D4F0E4E01213846FAF788FE0446AC42F1
:1068A00004D0FEF7D1FCB0EE408A07E0FEF7CCFC46
:1068B00030EE480A10EE100AB04201DC2546E9E746
:1068C000BDEC028BBDE8F081000002409A99993E30
:1068D000F8B5074600241D4E0FB1012300E0022346
:1068E000706904EB4405284402227821FFF7BAFCC2
:1068F0007169485D8000CD2210FB02F02944800AB6
:1069000048707169485D2944C0088870631CB3F5FC
:10691000966F16DAD6F814C0820805EB0C01487899
:1069200081081CF805008008FFF740FD00907169A0
:1069300003EB43000844BDF8001001809DF80210ED
:106940008170A41CB4F5966FC6DBF8BDE801002089
:1069500030B52DED028BADF51B7D64A090E80E10D7
:1069600045690469806999959592CDF85CC29894BF
:10697000969394919A90942263496FA8F9F750FCEA
:106980006822624955A8F9F74BFC582260493FA894
:10699000F9F746FCCC225F490CA8F9F741FC5EA050
:1069A00006AD90E80E1004694069A5E80E100A943F
:1069B0000B905FA001AC90E80E100069A4E80E10E7
:1069C0000590FDF78DFA0028FBD14EF66020FFF709
:1069D0004BFF00240025C823182294A95948FCF72E
:1069E0006BF8C82390226FA95648FCF765F800950C
:1069F00042F21073012269465248FBF79BFF9DF853
:106A00000000752802D06E2802D002E0012400E0C8
:106A10000124002CDFD0C823642255A94948FCF783
:106A20004BF8C82354223FA94648FCF745F89DF887
:106A3000000075280DD1C823CB220CA94148FCF7D2
:106A40003BF8C823102201A93E48FCF735F8FEF7B1
:106A500069FC9DF800006E280DD1C823162206A9F6
:106A60003848FCF729F8C823102201A93548FCF75B
:106A700023F8FEF73BFC3448FCF744FAFEF7E4FB4E
:106A8000B0EE408AFEF7E0FB30EE480A10EE100A46
:106A9000B0F1804F0CDAFFF7B1F9FFF7AFF9FEF76D
:106AA000D3FB30EE480A10EE100AB0F1804FF2DB53
:106AB0004FF4E130FCF726FAC82306222349244884
:106AC000FBF7FAFF234C01202070FDF709FA28B9E3
:106AD000FFF794F9FDF704FA0028F9D0022020709E
:106AE0000DF51B7DBDEC028B30BD00000D0A0D0ABB
:106AF00050617373207468727520555342206D6F16
:106B000064650D0A0000000008740008687500083C
:106B1000887300089C7400084E6F726D616C204D84
:106B20006F64652053656C65637465640D0A0000CD
:106B3000424F4F54494E47204D4F44554C450D0A46
:106B400000000000FC0500208024010061010020FD
:106B5000BC050020600100202DE9F047ADF5805D07
:106B60000746884692461E46E946202E14D84FF422
:106B7000626251464846F9F753FBCDF8206E39461C
:106B80004046FEF701FB40F624624946FEF704F951
:106B90000DF5805DBDE8F087002F39D00620FEF7A7
:106BA00027F80024C7F10105444519D0394620468D
:106BB000FEF7F2FAB0F1FF3F12D039462046FEF759
:106BC000E3FA01464FF480524846F9F729FBE9B24F
:106BD0002046FEF7D9FA4FF480524946FEF7DCF81A
:106BE000641C202CE0DB4FF4626251464846F9F702
:106BF00017FBCDF8206EE9B24046FEF7C5FA40F625
:106C000024624946FEF7C8F80DF5805DBDE8F087BF
:106C10000720FDF7EDFFC4E72DE9FF4F96B03D4E8D
:106C2000DFF8F4903378002B0DD1741C4FF0010C79
:106C3000E55C0CFA05F529F813505B1CDBB2202B40
:106C4000F6D386F800C00023DDF864C00DF1040817
:106C50000CEB4C0C0CEB0004641C48F82340B430E3
:106C60005B1CDBB2142BF5D38D1C961C4FF0000B74
:106C7000DFF8A8A0DE466C46199858443C2809D194
:106C8000002058F82010B43948F82010401CC0B239
:106C90001428F6D300278021ADF800E0ADF802E01B
:106CA000002058F8202012780A4209D01AF8002053
:106CB00039F810C034F8123043EA0C0324F81230CB
:106CC000401CC0B21428ECD3BDF800002880AD1DD4
:106CD000BDF802003080B61D49080029DCD1002033
:106CE0000F49C95758F820200A4448F82020401C72
:106CF000C0B21428F6D3781CC7B2032FCBD30BF144
:106D0000010000F0FF0BBBF13C0FB5D31AB0BDE89A
:106D1000F08F000018010020340200201302002030
:106D200010020020DFEDF70A20EE200ADFEDF60A60
:106D30004FF4B47180EE201ABDEEC10A10EE100AB5
:106D400090FBF1F201FB1200002801DA00F5B470AB
:106D5000EE495A2804DC01EB800090ED000A7047F0
:106D6000B42806DCC0F1B40001EB800090ED000A0D
:106D70007047B0F5877F07DCB43801EB800090EDF9
:106D8000000AB1EE400A7047A0F5B470A1EB800094
:106D900090ED000AB1EE400A7047DFEDDD0A30EEFB
:106DA000C00ABFE72DE9F74F04462DED020B2DED8C
:106DB0000E8B88B0B0EE408AF1EE00BACDED05BA88
:106DC000CDED04BA4FF0000BF3EE04EADFEDD1DABB
:106DD000B6EE00AA9FEDD00A28EE0ADAB7EE00EA76
:106DE00068EE00CA00EE10BAF8EE400A80EEAE0A75
:106DF0008DED030A4FF0000830EE4A0AF0EE6B0A00
:106E0000CBEB0B10069020EE80CA00EE108AF8EE55
:106E1000400A80EEAD0A8DED020A069808EB80006C
:106E200000EB400530EE4A0AF0EE6B1A61EE80AAE4
:106E3000B0EE6B2AF0EE4C8A3AEE880AFFF772FF4A
:106E4000F0EE402A38EE880A20EE0A0AFFF76AFFC1
:106E500070EE222A3AEEA80A30EE080A20EE0A0A5C
:106E6000FFF760FF30EE22BAB0EE6C0AFFF75AFF70
:106E700061EE8A0A40EE80AACDED00AAB0EE4D0A7E
:106E8000FFF78BFF62EE0A0A40EE808ACDED018AA1
:106E900018EE100AF9F7CBFB2AEEAA0A41EC190BFF
:106EA00008EEA80A30EE0E0A10EE100AF9F7BFFB42
:106EB00041EC100BFCF7B8FE53EC192B51EC100B06
:106EC000F9F7F0F9F9F7C6FB00EE100AFFF72AFF11
:106ED00030EE0B0A60EE0A1A199815286DD2DFE819
:106EE00000F06C0B3D3D0B6C6C6C6C6C6C6C3D5E27
:106EF0003D5E3D3D3D0B0B00DFED832A21EEA20AF6
:106F0000FFF710FF9FED852AF0EE420A40EE020ADD
:106F1000BCEEE00A10EE100AC6B29FED810A01EE47
:106F2000A20AFFF7FFFEF0EE420A40EE020ABCEEB4
:106F3000E00A10EE100A00F0FF0A9FED7A0A01EE57
:106F4000A20AFFF7EFFEF0EE420A40EE020ABCEEA4
:106F5000E00A10EE100A00F0FF092EE09FED6A0A29
:106F600021EE800AF0EE402AFFF7DCFE9FED6B2A4F
:106F7000F0EE420A40EE020ABCEEE00A10EE100A01
:106F8000C6B2B0EE620AFFF708FFF0EE420A40EE2A
:106F9000020ABCEEE00A10EE100AC7B20DE0DFED07
:106FA0005A0A9FED600A01EEA00AFFF7BBFEF0EE61
:106FB0004A0A40EE0A0ACDED000A1998152875D242
:106FC000DFE800F0B40B2B40235CB4B4B4B4B4B429
:106FD0004775558A324E39131B00681C6655411C93
:106FE00004F800A004F80190A6E0681C04F805A0CD
:106FF000411C265404F801909EE0681C04F805909A
:10700000411C04F800A0665496E0FF22681C6255FB
:10701000411C225404F801908EE0681C6655411C06
:1070200027540020605487E00021681C6155411CF2
:107030002754665480E0681C66550022411C225487
:10704000675479E0FF21681C6155411C2754665440
:1070500072E0681C6655FF22411C225467546BE0A5
:10706000681C6655411C2754FF20605464E0FF22D1
:10707000681C6255411C265462545DE09FED2A0A4B
:1070800021EE800AFFF74EFEF0EE400A9FED230A44
:10709000B0EE401A00EE801ABCEEC10A10EE100AE3
:1070A000691C60554A1C6054A05445E03EE09DEDCB
:1070B000000A681C60EE000A9DED1A0AB8EE400A4C
:1070C00020EE800ABCEEC00A10EE101A6155FF22B5
:1070D000411C225462542FE0FF22681C62559DED32
:1070E000000A411C60EE000A9DED1A0AB8EE400A43
:1070F00020EE800ABCEEC00A10EE103A235462540F
:107100001AE0000000003443DB0F49407402002005
:10711000DB0FC93F000070423BAAAA3E0000FF42BD
:10712000920A0640920A8640DB0F49418022681C81
:107130006255411C2254625408F10108B8F13C0F19
:10714000FFF463AE0BF1010BBBF1140FFFF44AAE79
:1071500008B00120BDEC0E8B05B0BDE8F08F4FF4F8
:1071600061635243120A521C91F800C00CFB02FCEE
:107170004FEA1C2C80F800C0401C491C5B1E002BF1
:10718000F2D170472DE9F0010B4600245243120A58
:107190000025561C4FF0000C00221F7893F8018048
:1071A000474493F80280C444BC441FFA8CFCDB1CA7
:1071B000521C3C2AF1DB0CFB06F2C2F30F22A24266
:1071C00000D914466D1C142DE4DB44F65852944249
:1071D0001ED900EE104ADFED100AB8EE400A80EE2C
:1071E000801ABCEEC10A10EE102A93B24FF461620D
:1071F00091F800C00CFB03FC4FEA1C2C80F800C087
:10720000491C401C521EF3D1BDE8F001012070471B
:10721000BDE8F0010020704700B09A4A0A01160646
:107220001702180B19031A0515041B0C1C011D0D60
:107230001E0B1F0E2010210F2211231224132514C0
:10724000262728292A2B2C2D2E2F30313233343566
:107250000909090909090D1A2830090909090A1F2C
:107260005083A7B50909090C3B91D6EFEBE1090959
:107270000C4AB8EED193624B090A3FBBEFA94917FC
:107280000A0709259AF0A733010101010F5BDFCE40
:10729000450A00A4C5C51F91F38B15080096F7F7A2
:1072A00030B5E959090800040D0D39C3DC42080165
:1072B0000086AEAE38C2DD440800009FE8E82EB17B
:1072C000EB5F0A0500040D0D1C88F2961908006A90
:1072D00099990D51D6D8540C01B4EEEE091D8AEEE1
:1072E000B94402050E0E090932A9F0BE60240F0848
:1072F00009090A39A3E9E1AE7F660909090A2B7970
:10730000C2E9F0EC0909090909163D6A8D9B0909D2
:10731000090909090A121C22000610160006101697
:10732000000000000102030401020304060708092B
:10733000000000000000E03F000000000000E0BF8F
:107340000000E0FE422EE63F0000E0FE422EE6BFD7
:10735000763C7935EF39EA3D763C7935EF39EABD4F
:107360003E5555555555C53F93BDBE166CC166BFBC
:107370002CDE25AF6A56113FF16BD2C541BDBBBEB5
:10738000D0A4BE726937663E546F206C6561766525
:107390002074686973206D6F64652C20707265734A
:1073A0007320616761696E2074686520626C756521
:1073B00020627574746F6E2C206F72207265736515
:1073C000742074686520626F6172642028626C6149
:1073D000636B20627574746F6E290D0A00000000E3
:1073E000415445300D0D0A0D0A4F4B0D0A000000A7
:1073F000434F4E4E4543540D0A0D0A4F4B0D0A00A4
:107400000D0A4F4B0D0A00005072657373202775EB
:107410002720666F7220626F6F74696E67207468D0
:1074200065204553503832363620696E20757067B6
:1074300072616465206D6F64652028666F722075C7
:107440007067726164696E672074686520666C613C
:107450007368206F66207468652045535038323653
:1074600036290D0A507265737320276E2720666FC8
:107470007220626F6F74696E67207468652045536F
:10748000503832363620696E207374616E646172D2
:1074900064206D6F64650D0A00000000466C617326
:1074A000682055706772616465206D6F6465207334
:1074B000656C65637465642E0D0A4E6F7720747970
:1074C0007065206120666577206B65797320696E31
:1074D000206F7264657220746F2068617665207415
:1074E0006865206D6F64756C6520746F20736574BA
:1074F00020697473206175746F20626175647261B4
:10750000746520746F2031313532303020626175FE
:1075100064730D0A5468656E20646973636F6E6EE0
:1075200065637420796F7572207465726D696E6120
:107530006C2066726F6D2074686520736572696176
:107540006C20706F72742C20616E642075736520DE
:1075500074686520466C617368446F776E6C6F6108
:1075600064546F6F6C0D0A000D0A596F75206172BB
:1075700065206E6F7720696E206469726563742080
:10758000636F6E6E656374696F6E207769746820CF
:1075900074686520455350383236362073657269F9
:1075A000616C206C696E6B2C207468727520796F29
:1075B00075722055534220706F7274204020313113
:1075C000353230302062617564730D0A00000000AE
:1075D00041542B43495041505F4355523D2231396C
:1075E000322E3136382E312E30222C223139322EA5
:1075F0003136382E312E30222C223235352E32358E
:10760000352E3235352E30220000000041542B43F8
:10761000575341505F4355523D224C4544545542C7
:1076200045222C22222C342C3000000041542B43C4
:10763000495053544152543D22554450222C22313A
:1076400039322E3136382E312E31222C3531323529
:107650002C353132352C300041542B4349504D5597
:10766000583D3000415445300000000041542B4348
:1076700057444843505F4355523D302C3100000081
:1076800041542B4349504D4F44453D3100000000CB
:1076900041542B43574D4F44455F4355523D3200B3
:1076A0004C4544545542453A4F46463A242400003E
:1076B0004C4544545542453A4D4F443A3F3F3F3F75
:1076C000242400004C4544545542453A494E543A0E
:1076D0003F3F3F3F242400004C4544545542453A27
:1076E0005350443A3F3F3F3F3F3F3F242400000078
:1076F0004C4544545542453A504F533A3F3F3F3F23
:107700003F3F3F24240000004C4544545542453A35
:107710005257433A000000004C4544545542453A04
:107720005241573A0000000048770008000000204E
:10773000E00300003C09000850790008E003002045
:1077400028160100003E00081102460132020A29F3
:107750000A086904092E38092A08093A0411201474
:10776000040102030504060806090C080F0A0E0DA1
:10777000030201000C230905070B0A0C070D0E0F6D
:107780000B19312117414141540D0A1364761B082E
:1077900090041A58041A0C041A6C0413D0751B08B0
:1077A0002C081A800413E07312080A1074045AF0AB
:1077B00018394CF11AF0381AD8041AB0041AC40453
:1077C0001318771B08A0081A08080110B2FFC2643A
:1077D000CB24F4282A02E839BE69731A010A190475
:1077E0002901390C014530757FF78E3C41F20E3D81
:1077F000465E563D3CDC8E3DD87EB23DC712D63D3E
:107800007496F93D5E830E3E3C30203EC8D0313E3A
:107810006F63433EE2E6543E8E59663E67BA773E5A
:10782000ED83843E4B208D3EC8B1953E7A379E3E17
:10783000D9B0A63E3F1DAF3E037CB73E7DCCBF3ED8
:10784000E50DC83ED53FD03E6361D83E2A72E03E8A
:107850006171E83EA25EF03E0439F83E18E13F88CF
:10786000D9033FC6A8073F766D0B3F46270F3FE081
:10787000D5123F1479163F8C101A3F069C1D3F1EEF
:107880001B213FC18D243F7CF3273F2B4C2B3F6CAA
:10789000972E3F1BD5313FF704353FAB26383F04C9
:1078A0003A3B3FC03E3E3FAD34413F761B443F0A2A
:1078B000F3463F17BB493F58734C3FBD1B4F3FF248
:1078C000B3513FD63B543F25B3563FAC19593F4CBB
:1078D0006F5B3FD0B35D3F19E75F3FE108623F094F
:1078E00019643F5D17663FCD03683F16DE693F3779
:1078F000A66B3FEE5B6D3F19FF6E3FB88F703F8800
:107900000D723F7978733F68D0743F4415763FED30
:1079100046773F5265783F5070793FE8677A3FE895
:107920004B7B3F611C7C3F1FD97C3F34827D3F7F76
:10793000177E3FFE987E3FA3067F3F5B607F50200F
:107940000B7F3F17D87F3F0AF67F3F0300803F0041
:04000005080001C529
:00000001FF
